:0200000480007A
:10000000B72F0000938F0F8073900F3015A8130047
:100010000000130000001300000013000000130094
:100020000000130000001300000013000000130084
:100030000000130000001300000013000000010086
:10004000970200009382020C73905230814001416C
:100050008141014281420143814301448144014580
:100060008145014681460147814701488148014950
:100070008149014A814A014B814B014C814C014D20
:10008000814D014E814E014F814F971102009381A6
:10009000E1D3170502001305E556979503009385F4
:1000A000257E01461122170502001305A548970574
:1000B0000200938565510146C52817A50300130565
:1000C000657C97B503009385A57B37B6ABAB13066C
:1000D000B6BAD92817B103001301C17AEF60F01343
:1000E000860293D21200F512638802008242110147
:1000F0006F00001073002030824211017300203025
:10010000711116C0F3222034E3CC02FC82421101AB
:10011000130141F806C20AC40EC612C816CA1ACC88
:100120001ECE22D026D22AD42ED632D836DA3ADCC7
:100130003EDEC2C0C6C2CAC4CEC6D2C8D6CADACC97
:10014000DECEE2D0E6D2EAD4EED6F2D8F6DAFADCA7
:10015000FEDE73252034F32510340A8601A07310C7
:10016000153492402241B2414242D2426243F243AC
:10017000025492542255B2554256D2566257F25703
:10018000064896482649B649464AD64A664BF64B33
:10019000065C965C265DB65D465ED65E665FF65F83
:1001A0001301C1077300203010C16374B50011053D
:1001B000E5BF828000000000000000000000000099
:1001C000000000000000000000000000000000002F
:1001D000000000000000000000000000000000001F
:1001E000000000000000000000000000000000000F
:1001F000197106C00AC20EC412C616C81ACA1ECC8D
:1002000022CE26D02AD22ED432D636D83ADA3EDCC6
:1002100042DEC6C0CAC2CEC4D2C6D6C8DACADECC96
:10022000E2CEE6D0EAD2EED4F2D6F6D8FADAFEDCA6
:100230009702020083A2423323A02200F32210344B
:1002400096DEEF00002B170102000321E13102418D
:10025000F65273901234B72200009382028873A082
:10026000023082403242C2425243E24372448254DC
:100270001255A2553256C2565257E2577258864806
:100280001649A649364AC64A564BE64B764C865C1A
:10029000165DA65D365EC65E565FE65F0961730059
:1002A0002030970202009382E23523A0120023A29D
:1002B000220023A4320023A6420023A8520023AA2E
:1002C000620023AC720023AE820023A0920223A21C
:1002D000A20223A4B20223A6C20223A8D20223AA06
:1002E000E20223ACF20223AE020323A0120523A2F2
:1002F000220523A4320523A6420523A8520523AADA
:10030000620523AC720523AE820523A0920723A2C7
:10031000A20723A4B20723A6C20723A8D20723AAB1
:10032000E20723ACF207EF409030170102000321EF
:10033000A1230241F65273901234B7220000938237
:10034000028873A0023082403242C2425243E243EA
:10035000724482541255A2553256C2565257E25731
:10036000725886481649A649364AC64A564BE64B45
:10037000764C865C165DA65D365EC65E565FE65FB1
:10038000096173002030970202009382A22783A0A4
:10039000020003A1420083A1820003A2C20083A243
:1003A000020103A3420183A3820103A4C20183A427
:1003B000020203A5420283A5820203A6C20283A60B
:1003C000020303A7420383A7820303A8C20383A8EF
:1003D000020403A9420483A9820403AAC20483AAD3
:1003E000020503AB420583AB820503ACC20583ACB7
:1003F000020603AD420683AD820603AEC20683AE9B
:10040000020703AFC20983AF820782807370043092
:10041000197106C00AC20EC412C616C81ACA1ECC6A
:1004200022CE26D02AD22ED432D636D83ADA3EDCA4
:1004300042DEC6C0CAC2CEC4D2C6D6C8DACADECC74
:10044000E2CEE6D0EAD2EED4F2D6F6D8FADAFEDC84
:100450009702020083A2421123A0220086DEEF2031
:10046000602E17010200032121100241F652739001
:100470001234B72200009382028873A002308240B7
:100480003242C2425243E243724482541255A25550
:100490003256C2565257E257725886481649A649F4
:1004A000364AC64A564BE64B764C865C165DA65DD0
:1004B000365EC65E565FE65F09617300203073707A
:1004C000043001A07310453082807325403073F0F2
:1004D00043308280970700009387A7FE232EB5FE46
:1004E0002322C5FA232635F82320F5F8130505F84D
:1004F0008280411106C6EF40B010EF10900A01E56E
:10050000B24041018280B24041016F20A023930795
:1005100085007D575CC118C55CC51CC9232005003A
:1005200082802328050082805C41DCC1984798C501
:1005300098474CC38CC788C91C4185071CC1828061
:100540009041FD57130785006314F60039A83E87D4
:100550005C439443E37DD6FEDCC18CC798C54CC395
:1005600088C91C4185071CC1828018495C43EDB7CE
:10057000584114451C4914C71845544154C3D84325
:100580006314A7001845D8C32328050088437D15A8
:1005900088C382803041AE8701CE4C455841B29528
:1005A0004CC563E4E5000C414CC53E856F30D02955
:1005B0008280411122C406C62A8426C2EF2030124E
:1005C0003C44635BF0025C5085CB9304440209A871
:1005D0003C44FD173CC43C446350F0025C5089CF5E
:1005E0002685EF2040586DD5EF2020783C44FD173C
:1005F0003CC43C44E344F0FEFD573CC4EF20701083
:10060000EF20F00D7C40635BF0021C4885CB930427
:10061000040109A87C40FD177CC07C406350F002B7
:100620001C4889CF2685EF2000546DD5EF20E0735C
:100630007C40FD177CC07C40E344F0FEFD577CC04D
:100640002244B240924441016F20B00B29CD0111E8
:1006500022CC2A8406CE26CA4AC84EC62E89EF204E
:10066000100824404C5C832904002685EF60801C20
:100670007D57232C0402B3079540CE974E9578C042
:1006800048C0232434015CC438C4631109021C48E7
:100690008DE7EF201007F2406244D2444249B2494C
:1006A0000545056182807370043001A013050401C3
:1006B000B93D13054402A13DE9BF13050401EF2034
:1006C000804A8547E317F5FC9133E1B701E5737084
:1006D000043001A0011126CA4AC84EC606CE22CC5B
:1006E000AA842E89B289A5C9EF60C01413055505E7
:1006F000EF30407D2A8435C5930745051CC144DC95
:1007000023202405EF20A07D24404C5C0329040015
:100710002685EF602012FD56232C0402B307954076
:100720003307A900CA9774C058C05CC434C4130509
:10073000040123242401E13B13054402C93BEF20BB
:10074000407C230834052285F2406244D244424969
:10075000B2490561828013054005EF30A0762A84F6
:1007600001E57370043001A000C051BF01E5737052
:10077000043001A06375B5007370043001A041110D
:1007800022C409462E84814506C6893711C500DD7D
:10079000B2402244410182807370043001A05D7137
:1007A00086C6A2C4A6C2CAC04EDE52DC56DA5AD8E9
:1007B0005ED632C6630A051C6382051C89476399AD
:1007C000F600585D85476305F7007370043001A09B
:1007D0003689AE842A84EF20C05B11E5B24781C719
:1007E0007370043001A0EF20806F185C5C5C014BDB
:1007F000894BFD59130A0401930A44026365F70CFF
:1008000063077919B2476381072463150B00280831
:10081000EF208048EF20E06EEF10604FEF20206C5B
:100820007C4063943701232204043C4463943701E1
:1008300023240404EF20E06C6C002808EF20E0473C
:10084000631E051EEF20A069185C5C5C630CF70A50
:10085000EF20206BEF20A0683C44634FF00039A8E4
:100860005685EF20403019C1EF2020503C44FD1741
:100870003CC43C446354F0005C50FDF32324340535
:10088000EF202068EF20A0657C40634FF00039A87E
:100890005285EF20402D19C1EF20204D7C40FD17DF
:1008A0007CC07C406354F0001C48FDF323223405D7
:1008B000EF202065EF10A06A054BEF204062185C26
:1008C0005C5CE37FF7F230406305060C631F09129E
:1008D0000844A685EF3040771C4434405840B69712
:1008E0001CC463EAE70A1C5C14405850850714C412
:1008F0001CDC5DC713054402EF20E0268547631129
:10090000F50AC9A8EF20E05FB2455285EF206007E5
:10091000EF20E05C3C44634FF00039A85685EF209F
:10092000802419C1EF2060443C44FD173CC43C4482
:100930006354F0005C50FDF323243405EF20605C29
:10094000EF20E0597C40634FF00039A85285EF203A
:10095000802119C1EF2060417C40FD177CC07C40A4
:100960006354F0001C48FDF323223405EF20605946
:10097000EF10E05E31F1593C054B81B73C41E38F0C
:1009800007E27370043001A07370043001A030409E
:1009900021E61C4085C71C5C585085071CDC39FBD0
:1009A000EF2020560545B640264496440649F259A4
:1009B000625AD25A425BB25B616182804840EF204A
:1009C00060491C5C58502322040085071CDCE3139B
:1009D00007F279D5253CE9B74844A685EF30C066D3
:1009E0003C4058441440B307F0403E9758C4637CE1
:1009F000D7025840BA975CC409475C506306E902C5
:100A0000185C050718DCC9DFF5B54844A685EF304A
:100A1000A0633C4058441440B307F0403E9758C48C
:100A2000E37CD7FCF9B75C50185C79DB185C7D1768
:100A300018DC185C050718DCA5D76DBD2285953E2E
:100A4000EF10E051014585B7EF20A04B0145A1BF54
:100A5000411126C2AA841305400522C406C6EF3000
:100A600060462A8415CD232C0502FD577CC105471D
:100A7000410558DC3CC42322040023200400232425
:100A80000400232604002320040423089404413492
:100A900013054402AD3C8146014681452285013360
:100AA0002285B24022449244410182800DC5411109
:100AB00022C426C206C64AC0032945002A84EF2064
:100AC000802C8144630CA900B2402244268502494F
:100AD0009244410182807370043001A05C448544DB
:100AE000FD175CC4F5F381460146814522854539F1
:100AF000E1BF31CDA1C9011122CC26CA4AC852C4D6
:100B000006CE4EC68947B68432892E8A2A846399D6
:100B1000F600585D8547630FF7047370043001A039
:100B20006D32185C5C5CAA896366F70281444E856D
:100B3000513AF240624426854249D244B249224A9F
:100B4000056182803C41C5DB7370043001A0737085
:100B5000043001A0304041E21C40D5CB1C5C7D57E5
:100B600085071CDC3C446387E7083C4485448507D3
:100B70003CC475BF993A185C5C5CAA89636DF70246
:100B8000304079DA4844D285EF30004C3C4058443C
:100B90001440B307F0403E9758C46375D7005840DF
:100BA000BA975CC48947E39BF4FA1C5CC5DB1C5C08
:100BB000FD171CDC65B7304045D24844D285EF3084
:100BC000A0483C4058441440B307F0403E9758C4F6
:100BD000E367D7FCD9BFDDF40844D285EF30C046C7
:100BE0001C4434405840B6971CC4E3E9E7F61C4067
:100BF0001CC4ADB75C5085449DDB13054402EF1067
:100C0000907615D5E30509F2232099000DB74840E9
:100C1000EF2040242322040091B721CD3C4181C71D
:100C20007370043001A01C41A1CB011122CC26CA53
:100C30002A844AC84EC606CE2E894138185C5C5CB0
:100C4000AA898144637DF7001C5C7D5785071CDC05
:100C50003C446388E7023C44854485073CC44E8598
:100C60009530F240624426854249D244B24905613A
:100C700082807370043001A05C41C5DB7370043066
:100C800001A05C5099E38544D9BF13054402EF10DD
:100C9000906D75D9E30909FE85472320F900E5B772
:100CA000397106DE22DC26DA4AD84ED652D456D224
:100CB00032C66302051C638A051AB68AAE892A8485
:100CC000EF20200D11E5B24781C77370043001A0F9
:100CD000EF20E0201C5C63920714B247638E070A82
:100CE0002808EF10707BFD5413094402130A040115
:100CF000EF202021EF10A001EF20601E7C406394C4
:100D00009700232204043C446394970023240404A2
:100D1000EF20201F6C002808EF10307A63130518AD
:100D2000EF20E01B1C5CADCFEF20A01DEF20201BAF
:100D30003C44634FF00039A84A85EF10D06219C1D6
:100D4000EF20A0023C44FD173CC43C446354F00037
:100D50005C50FDF324C4EF20C01AEF2040187C4003
:100D6000634FF00039A85285EF10F05F19C1EF1002
:100D7000D07F7C40FD177CC07C406354F0001C4851
:100D8000FDF364C0EF20E017EF10601DEF20201589
:100D90001C5CC1E7B247A9FFEF20A016014555A092
:100DA000EF2020161C40DDC7B2454A85EF10703D8C
:100DB000EF20E0123C44634FF00039A84A85EF1061
:100DC000905A19C1EF10707A3C44FD173CC43C4462
:100DD0006354F0005C50FDF324C4EF208012EF2038
:100DE00000107C40634FF00039A85285EF10B057D7
:100DF00019C1EF1090777C40FD177CC07C40635494
:100E0000F0001C48FDF364C0EF20A00FEF10201588
:100E100031C9EF20C00C1C5CB5DFCE85228544446F
:100E2000EFF04FF7639C0A041C5C1840FD171CDCB4
:100E300001E7EF20801148C01C48A1EFEF20600CB3
:100E40000545F2506254D2544259B259225A925A2C
:100E500021618280EF20A0084840EF109075EF20BC
:100E6000400A99B7EFF08FDA6DB73C41E38707E4AA
:100E70007370043001A07370043001A05C5044C44E
:100E8000D5DF13054402EF10104E4DD9EFF00FD807
:100E900075B713050401EF10104D8547E310F5FAFF
:100EA000F5B72285EFF0EFF0EF10600B014551BF71
:100EB0001DC9411122C44AC006C626C244412E891A
:100EC0002A84EF10506C6383A40281464A868145D0
:100ED0002285F93385476300F502B24022449244EB
:100EE0000249410182807370043001A05C440545D1
:100EF00085075CC4DDB75C4485075CC4F9BF15CDCC
:100F0000ADC9011122CC26CA4AC84EC652C42A8491
:100F100006CE3289AE89EFF04FDB1C5C2A8A814411
:100F200085E35285EFF00FDAF240624426854249AC
:100F3000D244B249224A056182807370043001A014
:100F4000304001CE4C445C40B2954CC463E4F500A3
:100F50000C404CC44E85EF30200F1C5C7D57FD17B4
:100F60001CDC7C40638CE7007C40854485077CC0AA
:100F70004DBF3C41D9D77370043001A01C4899E3A0
:100F8000854445B713050401EF10F03D75D9E30919
:100F900009FE85472320F900E5B721C93C41A1CDD1
:100FA000A1CB011122CC26CA4AC852C42A8406CE3B
:100FB0004EC62E8AEFF06FD11C5C2A89814491CBFA
:100FC0008329C400D2852285EFF0CFDC8544232617
:100FD00034014A85EFF00FCFF24062442685424942
:100FE000D244B249224A056182807370043001A064
:100FF0007370043001A0EDDF7370043001A001E5CF
:101000007370043001A0411122C42A8406C6EF1077
:10101000106D005CEF10F06EB24022852244410159
:10102000828001E57370043001A0411106C622C41C
:101030002A84EF10D06A1C5C405C1D8CEF10706C31
:101040002285B24022444101828019C1085D82801C
:101050007370043001A01DCD978703009387877EAE
:10106000D843630CE502D847630CE504D84B63070B
:10107000E504D84F6302E504D853630DE502D85761
:101080006308E502D85B6303E502D85F630EE50001
:101090006F2070757370043001A001470E07BA9776
:1010A00023A007006F2030741D47CDBF1947FDB73F
:1010B0001547EDB71147DDB70D47CDB70947F9BF64
:1010C0000547E9BF684582806CC5828003450505F8
:1010D000828009C5085D1335150082807370043065
:1010E00001A019C51C5D485D1D8D1335150082805A
:1010F0007370043001A0978703009387A774984307
:1011000005C3984705C7984B05C7984F05C798531F
:1011100005C7985705C7985B15C7985F15C38280A8
:1011200001470E07BA978CC3C8C382800547D5BF55
:101130000947C5BF0D47F5B71147E5B71547D5B7FF
:101140001D47C5B71947F1BF978703009387876F7E
:10115000D8436308E502D847630BE502D84B630A1E
:10116000E502D84F6309E502D8536308E502D85772
:101170006307E502D85B6308E502D85F6303A70253
:10118000828001470E07BA9723A007008280054797
:10119000D5BF0947C5BF0D47F5B71147E5B7154797
:1011A000D5B71D47C5B71947F1BF411122C426C2A3
:1011B0004AC02A8406C6AE843289EF105052784065
:1011C000FD576314F700232204043844FD576314C9
:1011D000F70023240404EF10D0521C5C99E74A86E0
:1011E000A68513054402EF10D00CEF10504F3C447D
:1011F000635BF0025C5085CB9304440209A83C4435
:10120000FD173CC43C446350F0025C5089CF2685F6
:10121000EF1070156DD5EF1050353C44FD173CC4F0
:101220003C44E344F0FEFD573CC4EF10904DEF10FA
:10123000104B7C40635BF0021C4885CB9304040197
:1012400009A87C40FD177CC07C406350F0021C481C
:1012500089CF2685EF1030116DD5EF1010317C400D
:10126000FD177CC07C40E344F0FEFD577CC0224467
:10127000B2409244024941016F10B0481DC17971DA
:101280004ECE52CC06D63E8A22D426D24AD056CA58
:101290005AC85EC6A547BA8963F8E7007370043080
:1012A00001A07370043001A02A8BAE843289B68B02
:1012B000C28A6307082213050006EF20B0402A8483
:1012C000630B05200A09232855034A869305500A13
:1012D0005685EF20706503C704001C587119230A56
:1012E000E40203C704003E991379C9FF79C783C795
:1012F0001400A30AF40283C71400E1C383C72400C7
:10130000230BF40283C72400CDCB83C73400A30B87
:10131000F40283C73400D5C383C74400230CF4020E
:1013200083C74400D9CB83C75400A30CF40283C7FE
:101330005400C1C783C76400230DF40283C764004F
:10134000ADCF83C77400A30DF40283C77400B5C783
:1013500083C78400230EF40283C78400B9CF83C7F8
:101360009400A30EF40283C79400A1CB83C7A4000A
:10137000230FF40283C7A400A9C383C7B400A30F3B
:10138000F40283C7B40095CB83C7C4002300F404E0
:1013900083C7C4009DC383C7D400A300F40483C7DC
:1013A000D40081CF83C7E4002301F40483C7E400A1
:1013B00089C783C7F400A301F404930A4400568547
:1013C000A30104042326340323283405232A040418
:1013D000EFF02F9513058401EFF0AF94A947B38781
:1013E0003741232C040400C81CCC40D02322040421
:1013F000232E04045E86DA854A85EFF0AF8D08C09F
:1014000063040A0023208A007370043017F9010076
:101410001309C9138327090097F401009384C414A6
:1014200091C798409C407C4385077CC317F7010017
:10143000130787121C43850797F6010023AEF610A9
:101440009C40C5CB8327090017FB0100130B4B23DE
:1014500089EB9C40DC5763E6F90097F7010023A570
:10146000871097F701009387670D9C4317F70100DA
:101470001307070E48541843850797F6010023AF5A
:10148000F60A3CC46376A70097F7010023A2A70CD5
:10149000D145EF50203AD6855A95EFF0EF88832753
:1014A000090081C79C40FC43B5E38327090005443C
:1014B00099C79C40DC5763F43701EFE03FF5228584
:1014C000B250225492540259F249624AD24A424BD3
:1014D000B24B456182805685EF20F0307D54C5B710
:1014E00013152600EF20101EAA8AE31605DC7D5492
:1014F000F9B797F7010023A98706184385476301C9
:10150000F70217FB0100130BAB17A1BF98409440E3
:101510007C43FD177CC3FC42C9FB7360043071B788
:10152000014A17FB0100130BAB15A94B5285D1459E
:10153000EF504030050A5A95EFE07FFDE3187AFF3F
:1015400097FB0100938B4B205E85EFE05FFC17FA61
:101550000100130AAA205285EFE07FFB17F5010076
:1015600013050521EFE0BFFA17F5010013058521EA
:10157000EFE0FFF917F5010013050522EFE03FF951
:1015800097F7010023A077FF97F7010023AA47FDF3
:10159000C9BD411122C406C626C24AC02A8473703E
:1015A000043097F40100938464FA9C40F9E311E459
:1015B00097F70100938747FB8043130944004A854E
:1015C000EFE01FFB1C5489C713058401EFE05FFAAD
:1015D000CA8517F501001305E51AEFE0FFF497F748
:1015E00001009387A7F7984397F70100938707F5C2
:1015F0009C43050797F6010023A2E6F6984085076D
:1016000097F6010023ACF6F201CB97F70100938720
:10161000A7F59843784349EF9C40B1C797F701007D
:10162000938787F49843630F87087370043098405A
:1016300039EB17F701001307E7F214439442A5E2D0
:101640007D5797F6010023A9E6EE984009CF98430D
:10165000784311CB984394437C43FD177CC3FC42F1
:1016600099E373600430B24022449244024941013C
:10167000828097F70100938727EF98439C437C4330
:1016800085077CC32DB794439843F8420507F8C2F9
:1016900017F70100130707ED14439442D5D21843FE
:1016A00058475847584397F6010023A7E6E871BF0B
:1016B000984394437C43FD177CC3FC42B1FF7360A5
:1016C000043099BF97F701009387C7E69C4381C711
:1016D0007370043001A02244B24092440249410197
:1016E0006FE0DFD241C517F701001307E7E71443A6
:1016F0008147638BA606411106C622C426C27370B9
:10170000043097F60100938666E49C4291C710432B
:101710001C437C4285077CC29C42AA84404981C705
:101720001C43FC43B9E797F701009387A7E39C4369
:10173000638B870497F70100938787E29C43638458
:10174000870497F70100938727056309F40297F749
:101750000100938727036301F4028547B2402244C6
:1017600092443E85410182803E85828073700430C0
:1017700001A0EF50E01F45BF9147CDB79C5493B7F0
:1017800017008907E1BF8947D1BF7370043097F70D
:1017900001009387A7DB984309EF15C59C43485583
:1017A00081CB97F70100938727DC9843784315E3B3
:1017B000828017F70100130727DB14431843F84210
:1017C0000507F8C261FD17F701001307E7D90843C1
:1017D000F1B7984394437C43FD177CC3FC42E9FB7B
:1017E000736004308280411122C42A8406C6EFE06F
:1017F000DFCD11E497F70100938707D7804340546A
:10180000EFE05FCCB2402285224441018280A547AF
:1018100063F5B7007370043001A0011122CC06CE2D
:1018200026CA4AC84EC652C42A847370043017F9B7
:1018300001001309A9D183270900CDEF71C43C48E9
:101840006388F50817F70100130707D263FCB70098
:101850001443638C860C18434457B3B4950093C467
:10186000140029A00443818C93B41400585463835A
:10187000E70A1C4C2CC863C60700A947B385B740CC
:101880000CCC93172700BA97584897F90100938911
:1018900029DF8A07CE97631AF702130A440052859C
:1018A000EFE01FCD97F70100938787CA48549C4308
:1018B00063F6A70097F7010023ACA7C8D145EF4016
:1018C0007077D2854E95EFE03FC699C0EFE01FB428
:1018D0008327090081CB97F701009387E7C89C43D2
:1018E000FC439DEBF2406244D2444249B249224A51
:1018F0000561828097F70100938707C798439C434F
:101900007C4385077CC305FC97F701009387C7C517
:10191000804335B74CD4B1BF6244F240D24442490F
:10192000B249224A05616F50A004814481B725C1A4
:10193000011126CA97F40100938404C39C4006CE8B
:1019400022CC4AC84EC6638DA7027370043017F9C3
:1019500001001309A9BF8327090091C798409C4043
:101960007C4385077CC3584997F701009387C7E2FA
:101970006302F7028327090081C79C40FC43A5EB63
:10198000F2406244D2444249B24905618280737098
:10199000043001A01C5517F70100130767DDE38B26
:1019A000E7FCE9FB930945002A844E85EFE05FBC24
:1019B00097F701009387C7B948549C4363F6A70083
:1019C00097F7010023A6A7B8D145EF40B06697F777
:1019D00001009387E7CA3E95CE85EFE0FFB49C40B7
:1019E0005854DC57E368F7F8EFE05FA261B7624450
:1019F000F240D2444249B24905616F40707715CD3B
:101A0000011122CC26CA4EC62A8406CE4AC8EFE06F
:101A1000DFAB584897F70100938707D8AA8981441C
:101A20006300F7024E85EFE0FFA9F240624426858D
:101A30004249D244B249056182807370043001A0EA
:101A40001C5417F501001305A5D2E38DA7FCF9FB83
:101A500097F70100938707AE9C43A9EB97F7010026
:101A6000938787B09C43445413094400DC574A854C
:101A7000B3B4F400EFE0DFAF97F70100938747AD11
:101A800048549C4393C4140063F6A70097F70100E1
:101A900023A0A7ACD145EF40F05997F701009387F9
:101AA00027BECA853E95EFE03FA8ADBF93058401F0
:101AB000EFE09FA785BF0111056506CE22CC26CA9F
:101AC0004AC84EC652C456C25AC0EF20A03F630E49
:101AD000051AAA8413050006EF20C03E2A84630A73
:101AE000051C05669305500A04D92685EF20C063BE
:101AF00004588567F117BE94B7474C4593879744C0
:101B0000130A44005CD85285230C0402A301040488
:101B10002326040223280404232A0404EFE07FA0E0
:101B200013058401EFE0FF9FA947232C0404F198DB
:101B300000C81CCC40D023220404232E04040146F8
:101B4000971500009385E5B12685EFE0BF9808C0A2
:101B50007370043017F901001309499F83270900A6
:101B600097F40100938444A091C798409C407C4323
:101B700085077CC317F701001307079E1C438507E1
:101B800097F6010023AAF69C9C40C9C3832709004D
:101B900097F901009389C9AE81EB9C40DC5789E736
:101BA00097F7010023A2879C97F701009387079975
:101BB000984397F601009386A6995C5494420507D2
:101BC00017F60100232CE69638C463F6F60017F7E3
:101BD0000100232FF796139527003E950A05D2851D
:101BE0004E95EFE07F948327090081C79C40FC431A
:101BF000DDE78327090091C39C40EF10704A8547B9
:101C00006305F50C59E17370043001A097F70100EA
:101C100023AC87941843854797F90100938949A617
:101C2000E314F7F8CE8A17FB0100130BEBB15685CE
:101C3000D10AEFE0DF8DE31C5BFF17F50100130510
:101C4000A5B0EFE0DF8C97FA0100938A2AB15685A0
:101C5000EFE0FF8B17F50100130585B1EFE03F8B37
:101C600017F50100130505B2EFE07F8A17F50100B3
:101C7000130585B2EFE0BF8997F7010023A4678FB2
:101C800097F7010023AE578D05B7F2406244D24466
:101C90004249B249224A924A024B056182809840E9
:101CA00094407C43FD177CC3FC42A1F77360043071
:101CB00089B76244F2404249B249224A924A024BF1
:101CC0002685D24405616F20003273700430FD57C1
:101CD00017F701002322F786624497F7010023A734
:101CE000A786F240D2444249B249224A924A024B64
:101CF00097F7010023A0078605616FE08FDA737004
:101D0000043097F7010023A307846FE0CFE717F7AC
:101D10000100130727821C4385071CC38280737050
:101D2000043097F7010093876782984305E317F71C
:101D300001001307278208439C4381CB97F70100DA
:101D4000938787829843784301EF828017F70100D9
:101D50001307878114431843F8420507F8C2C1BF2F
:101D6000984394437C43FD177CC3FC42F9FF7360A6
:101D700004308280411106C622C4EFE00FF597E7D8
:101D800001009387277D8043EFE0CFF3B2402285A7
:101D900022444101828097E701009387E77B8843D3
:101DA0008280797106D622D426D24AD04ECE52CC29
:101DB00056CA5AC85EC697E701009387A7779C4327
:101DC000B1EF17E701001307E7781C43850797E693
:101DD000010023A1F678832A0700638F0A0697E79C
:101DE0000100938767759C43814463F1FA0897F972
:101DF00001009389E98817EA0100130AEA7683272C
:101E00000A008546D85793172700BA978A07BE99C4
:101E100083A7090063FFF600854421A897E7010026
:101E2000938787729C438144850717E70100232D20
:101E3000F77097E701009387E7709C4391C385444F
:101E4000B2502254268502599254F249624AD24A2B
:101E5000424BB24B4561828017E401001304847049
:101E60001C409C43DDC37370043001A017E40100E3
:101E70001304446F97F901009389898017EA0100E0
:101E8000130A8A6E17EB0100130B8B6C1C409C43EA
:101E9000B5C31C40DC4703A9C70083274900930B47
:101EA00049005E8563EEFA04EFE08FEC8327890238
:101EB0001305890199C3EFE0AFEB8327C90203271C
:101EC0000B00DE85139527003E950A054E95637637
:101ED000F70017E70100232DF766EFE0EFE4832713
:101EE0000A000327C902DC57E362F7FA1C40854465
:101EF0009C43C5F3FD5717E70100232FF76201B795
:101F000017E70100232AF762DDBD17E70100130779
:101F100027651C40184397E6010023A5E66417E7F0
:101F20000100232FF76297E70100938767619C43C5
:101F3000850717E701002325F7601C409C4399E7BC
:101F4000FD5717E701002329F75E51BD1C40DC4710
:101F5000DC47DC4317E701002320F75E49B597E72C
:101F600001009387275D984301E77370043001A057
:101F7000011106CE22CC26CA4AC84EC652C456C249
:101F80005AC07370043097E401009384245C984035
:101F900061EB98437D1797E6010023ADE6589C431B
:101FA000D9EB97E701009387275B9C43C9C797EA62
:101FB0000100938AEA6C17EA0100130A6A5917E9CB
:101FC00001001309695A854919A83385EA00EFE031
:101FD000AFD5832709005854DC576379F70483A7EA
:101FE0000A0FC1CF83A7CA0FC04713058401EFE0D2
:101FF0002FD8130B44005A85EFE08FD75C5483260B
:102000000A00DA85139527003E950A052A8756951A
:10201000E3FDF6FA17E70100232CF752EFE0CFD0EB
:10202000832709005854DC57E36BF7FA97E7010060
:1020300023AA37516DB701449C4081CB97E701003B
:10204000938787529C43FC4395E72285F240624484
:10205000D2444249B249224A924A024B05618280E7
:1020600017E701001307475014431843F8420507C8
:10207000F8C205B7EF40D00FC9BF17E40100130441
:10208000A44C1C4095C31C40054999CF193B09C578
:1020900097E7010023A8274B1C40FD1717E7010015
:1020A0002324F74A1C40FDF397E7010093878749F3
:1020B00098438547E311F7F8EFE04FB50544ADBF0E
:1020C00011CD81E57370043001A017E701001307FB
:1020D00067461C4399C77370043001A073700430C5
:1020E00001A0411122C406C614431841850617E613
:1020F00001002321D64497E601009386A645944229
:102100003304B70000C163F7E602637FE40063FDB8
:10211000860097E701009387274588431105EFE084
:102120002FC52285EF40807E1D3D01C9B24022446B
:1021300041018280E36FE4FCD9BF2244B2404101F7
:102140006FE0CFAC11C917E701001307A73E1C438E
:1021500091C77370043001A06FE04FAB411106C608
:1021600022C41843AA87050797E6010023A4E63C8A
:1021700097E601009386463F17E701001307873D66
:10218000184388423304F7001105EFE06FBE228543
:10219000EF40C077E93311E52244B24041016FE0DE
:1021A000EFA6B240224441018280411122C406C6FA
:1021B00097E70100938707389C430144850717E799
:1021C00001002329F73697E701009387E7389C43FE
:1021D00063E0F51217EE0100130E4E5697E2010070
:1021E0009382424901440147854F1303500A21A0BD
:1021F000311E638DC20B83278EFFBA86F5DB8327E2
:10220000CEFFDC43232EFEFE638AC70F03AFC70059
:10221000DC432A97814E232EFEFE6385C70783A8E1
:10222000C70093874803232017015CC383A7880452
:102230002326F7011CC783A7C8021CCB83A7080568
:10224000232C07005CCB03A8080383470800639096
:102250006704C287850783C60700B3850741E38B00
:1022600066FE8981C205C181231EB700850E130752
:10227000070263061F038327CEFFDC43232EFEFEE7
:10228000E39FC7F983274E00232EFEFE49BF8145F9
:10229000231EB700850E13070702E31E1FFD769469
:1022A00013175400311EBA86E397C2F597E7010071
:1022B0009387472B03AE070083270E00639D070E0D
:1022C00097E701009387C72903AE070083270E0015
:1022D0006392071817EE0100130E8E3A83274E10F3
:1022E0009DE383278E116395072019C223200600E2
:1022F000BD312285B24022444101828083274E00B5
:10230000232EFEFE21B783278E1017EF0100130F37
:10231000EF47DC4317E701002328F7466380E733E4
:1023200083A2C700DC43AA96814E17E70100232D44
:10233000F744914F1303500A6388E70783A8C70047
:102340009387480323A01601DCC283A7880423A631
:10235000F6019CC683A7C8029CCA83A7080523ACC4
:102360000600DCCA03A80803834708006391672AB4
:10237000C287850703C70700B3850741E30B67FEE4
:1023800093D72500C207C183239EF600850E93864E
:1023900006026386122983278E10DC4317E70100AB
:1023A0002324F73EE39CE7F983270E1117E701008A
:1023B000232CF73C61B783274E00130F8E00D443C4
:1023C0002322DE006388E629B307E500D84283A212
:1023D000C600814E2322EE00894F1303500A630684
:1023E000EF068328C7001387480323A01701D8C32B
:1023F00003A7880423A6F70198C703A7C80298CBB0
:1024000003A7080523AC0700D8CB03A8080303479C
:1024100008006318671C4287050783460700B30559
:102420000741E38B66FE13D7250042074183239EB5
:10243000E700850E93870702638D121B83264E00EB
:10244000D8422322EE00E31EEFF80327CE0023221A
:10245000EE0041BF83274E00130F8E00DC43232282
:10246000FE006384E71F83A2C700DC43AA96814E67
:102470002322FE00894F1303500A6306FF0683A838
:10248000C7009387480323A01601DCC283A78804F2
:1024900023A6F6019CC683A7C8029CCA83A7080589
:1024A00023AC0600DCCA03A8080383470800639630
:1024B0006710C287850703C70700B3850741E30B91
:1024C00067FE93D72500C207C183239EF600850EC1
:1024D00093860602638B120F83274E00DC43232270
:1024E000FE00E31EFFF88327CE002322FE0041BF3B
:1024F0008327CE1197EE0100938E8E2ADC4317E7D7
:102500000100232DF7286384D71383AFC700DC4372
:102510003307D500014397E6010023A1F6280D4FAC
:1025200089429308500A6387D707C8479307450332
:1025300008C35CC33C452326E7011CC75C551CCB84
:102540001C5599C3232657003C49232C07005CCB1C
:10255000032805038347080063951705C28785078D
:1025600083C60700B3850741E38B16FF93D7250089
:10257000C207C183231EF700050313070702638AFE
:10258000AF028327CE11DC4397E6010023A8F62093
:10259000E39DD7F983274E1297E6010023A0F6208A
:1025A00069B78147231EF700050313070702E39A63
:1025B000AFFC1A94E31C06D225BB8147239EF6008C
:1025C000850E93860602E39912F117EE0100130EB1
:1025D0002E0B83274E10769493165400E38307D076
:1025E0001DB30147239EE700850E93870702E397FB
:1025F00012E597E701009387A7F603AE07007694EC
:102600009316540083270E00E38607CCA1B58147BB
:10261000239EF600850E93860602E39E12D783273B
:102620008E11769493165400E38107CCD1B583279D
:102630004E1217E701002323F716C1BD83270E11A1
:1026400017E701002322F714E1B98327CE002322E4
:10265000FE0011BD8326CE002322DE00B5B37971C2
:1026600026D24AD04ECE52CC56CA5AC85EC606D6DC
:1026700022D497E901009389E9EB17E901001309D6
:10268000290017EA0100130A6AEC97EA0100938A0D
:10269000AAED97EB0100938B2BEC97E40100938458
:1026A000E4EB054B21A883A7090003244910850703
:1026B00017E701002320F7E85D3011E89C40E5F7BB
:1026C00083270900E37CFBFEEFD05FD4C5BF7370A6
:1026D000043083270A00B9E383270911C047130593
:1026E0004400EFD0FFE883A70B00FD1717E70100B8
:1026F0002324F7E69C40FD1717E701002320F7E6A7
:1027000083270A0089C783A70A00FC4385E308588A
:10271000EF10700D2285EF10100D4DB703A70A00C2
:1027200083A70A007C4385077CC37DB703A70A0003
:1027300083A60A007C43FD177CC3FC42E9FB73605F
:102740000430F1B797E701009387C7DE9C43DDE7CC
:10275000411106C622C426C297E7010023A407DE62
:1027600017E70100130747E01C43B7A6A5A593860A
:10277000565A9C5B8C43639BD500D0436318B600CC
:1027800094476395C600DC476388D70008430C4331
:1027900093854503EF20B00217E70100130747DBDD
:1027A000144317E401001304A4ED11A81C43A9CF9E
:1027B0001C43FD1797E6010023ACF6D8144393970A
:1027C0002600B6978A07A2979C43EDD30843931738
:1027D0002500AA978A073307F4005443A107A2975C
:1027E000C44244C36385F402DC44B240224417E788
:1027F0000100232BF7D6924441018280854717E7D9
:1028000001002321F7D482807370043001A0C440FA
:10281000D145EF402002229544C1F9B701114AC8C1
:1028200006CE22CC26CA4EC62A897370043097E49D
:1028300001009384A4D19C4017E401001304C4D286
:10284000D9E76314090003290400930949004E8560
:10285000EFD01FD28327890289C713058901EFD0E2
:102860003FD1CE8517E50100130505F3EFD0DFCB8F
:102870009C4081C71C40FC43ADE31C40638B270791
:102880009C409DCF737004309C40C1EB97E70100E2
:10289000938747CD9843184325EBFD5717E7010071
:1028A000232CF7C89C4089CF1C40FC4391CB184097
:1028B00014407C43FD177CC3FC4299E373600430F1
:1028C000F2406244D2444249B249056182801840D4
:1028D0001C407C4385077CC3ADB7184014407C4343
:1028E000FD177CC3FC42D1FB736004301C40E399AC
:1028F00027F99C40A1C397E701009387A7C39C4396
:10290000ADCB7370043001A09C43DC47DC47DC4353
:1029100017E701002322F7C271B718401C407C431F
:1029200085077CC397E701009387C7C39843184383
:102930002DD7D9BF97E70100938707C217E701009A
:10294000130707D49C4303278711631DF700F24048
:10295000624497E7010023A907C0D2444249B24923
:10296000056182806244F240D2444249B249056125
:10297000D1BB6244F240D2444249B24905616FD0B2
:10298000FFA83DC9411126C297E401009384C4BD4C
:102990004AC02E898C4006C622C4E105EFD05FBA3A
:1029A00088401105EFD0DFBCFD57630AF90497E7B3
:1029B0000100938727BA804398409C434A9440C3C0
:1029C000636CF40497E701009387C7B988438C4090
:1029D0009105EFD0FFB697E701009387E7B59C43D9
:1029E0006376F40097E7010023A887B4B24022443D
:1029F00092440249410182807370043001A08C40EE
:102A00002244B2409244024917E501001305C5D89B
:102A1000910541016FD05FB197E70100938747B4FB
:102A2000884322448C40B2409244024991054101BE
:102A30006FD01FB111C997E701009387A7AF9C43DF
:102A400099E77370043001A07370043001A0411144
:102A500026C297E40100938424B19840AE878C404D
:102A6000B7060080D58F06C622C41CCFE10532848C
:102A7000EFD09FAB88401105EFD09FAFFD57630E9D
:102A8000F40097E701009387E7AC8843B240924493
:102A90002295224441016F3070678C402244B2403D
:102AA000924417E50100130525CF910541016FD030
:102AB000BFA725CD411126C297E401009384C4AA83
:102AC0004AC02E898C4006C622C4E1053284EFD06C
:102AD000BFA588401105EFD0BFA98547630AF4045C
:102AE00097E70100938707A7804398409C434A9447
:102AF00040C3636CF40497E701009387A7A688435B
:102B00008C409105EFD0DFA397E701009387C7A220
:102B10009C436376F40097E7010023AF87A0B2409F
:102B2000224492440249410182807370043001A022
:102B30008C402244B2409244024917E5010013053B
:102B4000A5C5910541016FD03F9E97E7010093878E
:102B500027A1884322448C40B24092440249910507
:102B600041016FD0FF9D411106C622C426C25C45BB
:102B7000C04735CC930484012685EFD07F9F97E72B
:102B800001009387279B9C43B5E793044400268567
:102B9000EFD01F9E97E701009387879B58549C4373
:102BA00063F6E70097E7010023A4E79A931727004D
:102BB000BA978A0717E50100130585ACA6853E95EF
:102BC000EFD09F9697E701009387079A9C4358544C
:102BD0000145DC5763F8E700854717E70100232329
:102BE000F7960545B24022449244410182807370B9
:102BF000043001A0A68517E50100130565B7EFD0E5
:102C0000BF92C9B797E701009387C7929C4381E7BA
:102C10007370043001A0411106C622C426C2B70752
:102C200000804045CD8F1CC12DC4EFD07F9493040C
:102C300044002685EFD0DF9397E701009387479103
:102C400058549C4363F6E70097E7010023A2E790FE
:102C500093172700BA978A0717E50100130545A2C5
:102C60003E95A685EFD05F8C97E701009387C78FCD
:102C70009C4358540145DC5763F8E700854717E744
:102C800001002321F78C0545B240224492444101C2
:102C900082807370043001A011CD97E70100938703
:102CA000278A984397E701009387C78A9C4318C1F6
:102CB0005CC182807370043001A055C1D1CD411137
:102CC00006C622C42A877370043097E801009388EF
:102CD000E88783A7080091CB97E701009387C7880F
:102CE00094439C43FC428507FCC217E30100130395
:102CF00063869C4103260300FD560144638FD7027F
:102D000017EE0100130ECE8303250E0003280700E3
:102D100054436305A80005446371D6023308D640C6
:102D20000544637CF80003250E00918F0326030001
:102D3000B6979CC108C350C3014483A7080081CB48
:102D400097E70100938747829C43FC4381EF2285EC
:102D5000B2402244410182807370043001A073703C
:102D6000043001A0EF30D040DDB7854717D7010010
:102D7000232AF77C828019C16845828001458280C0
:102D800011C16CC5828097D701009387E77D884386
:102D9000828097D701009387677B9C43054589CB49
:102DA00097D70100938707798843133515000605E7
:102DB000828031CD011126CA97D401009384C47A50
:102DC0009C4006CE22CC4AC84EC65855DC57637983
:102DD000F7021C4D63C707009C40D457A947958F45
:102DE0001CCD93172700BA97584917E9010013091A
:102DF00029898A07CA97630DF7009C40DC575CD588
:102E0000F2406244D2444249B249056182808280E4
:102E1000930945002A844E85EFD08FF59C4017D743
:102E200001001307E7721843DC575CD46376F700A0
:102E300017D70100232EF770139527003E956244A3
:102E40000A05F240D244CE854A95B249424905610D
:102E50006FD08FED19CD411106C622C426C297D777
:102E600001009387677080436307A4007370043088
:102E700001A0014582807C4881E77370043001A085
:102E800054543848FD177CC86383E60099C7014550
:102E9000B24022449244410182809304440026853A
:102EA000EFD00FED284897D701009387676A9843C2
:102EB000A947898F48D41CCC6376A70097D7010017
:102EC00023A8A768D145EF30F01697D70100938764
:102ED000277B3E95A685EFD02FE5054555BF73703E
:102EE000043097D70100938767669C4391CB97D7AF
:102EF00001009387676798439C437C4385077CC3A5
:102F0000828097D70100938767649C438DC397D7CE
:102F10000100938767659843784311CB98439443A6
:102F20007C43FD177CC3FC4299E3736004308280CC
:102F300097D7010093874763904394439843A947E9
:102F4000D456084E958F1CCF828097D70100938767
:102F5000A761984309C79443F84A0507F8CA88430C
:102F6000828079714AD006D622D426D24ECE2A89C2
:102F70007370043097D401009384445D9C4017D44F
:102F800001001304645EBDE31C40BC4F89E71C4094
:102F90000547F8CFD1E19C4081C71C40FC43F1EBD1
:102FA000737004309C408DEF1C40A84F11C5630422
:102FB00009021C4023AC07041C4023AE07049C40BC
:102FC00081C71C40FC438DEBB250225492540259ED
:102FD000F2494561828018403C4FFD173CCFE9BF64
:102FE00018401C407C4385077CC37DBF18401C40B3
:102FF0007C4385077CC349BF184014407C43FD17C0
:103000007CC3FC42F1F373600430B25022549254FA
:103010000259F2494561828008402EC61105EFD061
:103020002FD5B245FD576380F50697D701009387EA
:10303000675283A9070018409C43AE9923223701A9
:1030400063ECF90497D701009387C75188430C407C
:103050009105EFD0EFCE97D701009387E74D9C43C2
:1030600063F6F90097D7010023A8374DEFD00FBAC8
:103070001DB7184014407C43FD177CC3FC428DF300
:103080007360043031BF0C4017D501001305C570C3
:103090009105EFD06FC9D9BF97D701009387474CEF
:1030A00088430C409105EFD0AFC9C9B779714AD0B8
:1030B0004ECE06D622D426D252CC2E89B289737037
:1030C000043097D40100938464489C4017D40100D5
:1030D00013048449F9EF18408947784F630CF700CF
:1030E0001C401345F5FFB84F798DA8CF1C4005470C
:1030F000F8CFADE69C4081C71C40FC43F5E37370FC
:1031000004309C40B1E7638609001C40BC4F23A0FB
:10311000F900184085470145784F630BF7001C40C4
:103120001349F9FF0545B84F3379E90023AC27056A
:103130001C4023AE07049C4081C71C40FC43C1E3F4
:10314000B250225492540259F249624A4561828037
:1031500018401C407C4385077CC375B7084036C6C1
:103160001105EFD0EFC0B246FD576385F60897D73B
:1031700001009387273E03AA070018409C43369A14
:10318000232247016363FA0897D701009387873D9D
:1031900088430C409105EFD0AFBA97D701009387D1
:1031A000A7399C436370FA0697D7010023A64739D5
:1031B00091A818401C407C4385077CC329BF184058
:1031C00014407C43FD177CC3FC42BDFB736004309C
:1031D000B250225492540259F249624A45618280A7
:1031E000184014407C43FD177CC3FC4289FB73608C
:1031F000043031B70C4017D501001305E55991058E
:10320000EFD08FB2EFD08FA0F5B597D7010093879D
:10321000273588430C409105EFD08FB2E5B751C1F7
:10322000411106C622C426C24AC07370043097D426
:1032300001009384A4319C40B9EB99C23C4D9CC2DF
:10324000B2878946704D74CD2E872A846386D7064F
:1032500063FCF6048D456387B70091456395B7001D
:103260006300D60C38CC8547630FF60405449C40B8
:1032700081CB97D701009387272F9C43FC43A9E379
:103280002285B2402244924402494101828097D76C
:1032900001009387672D98439C437C4385077CC33B
:1032A00069BF7370043001A08546E39ED7FA3C4D98
:1032B00033E7B70038CD45BF3C4D85073CCD65B7FA
:1032C000EF30006B75BF130944004A85EFD04FAA59
:1032D00097D701009387C72748549C4363F6A700FC
:1032E00097D7010023A6A726D145EF30A05497D742
:1032F00001009387E7383E95CA85EFD0EFA21C54B2
:1033000081C77370043001A097D701009387C72548
:103310009C435854DC57E3FBE7F4EFD02F8FB9B749
:103320000144B1B739CD011122CC26CA4AC84EC6D4
:1033300052C456C206CEBA89368AB2842E892A84ED
:10334000EFD0AF98AA8A63050A003C4C2320FA000C
:10335000784C89477CCC6389F40263F4970C8D46E2
:103360006387D40091466396D400630AF70A232C3E
:1033700024058547631EF7061C5499CB73700430EF
:1033800001A07370043001A03C4C85073CCCD5B73C
:1033900097D701009387071A9C43ADEB9304440031
:1033A0002685EFD0EF9C97D701009387671A485482
:1033B0009C4363F6A70097D7010023ABA718D1451C
:1033C000EF30404797D701009387872BA6853E951E
:1033D000EFD08F9597D70100938707199C435854D6
:1033E000DC5763F7E70063850900854723A0F900F0
:1033F00005445685EFD00F8D2285F2406244D244B9
:103400004249B249224A924A056182809305840169
:1034100017D501001305C535EFD00F9165BF0144E5
:10342000C9BF8547E397F4F43C4C33E92701232CCB
:10343000240581B74DC1011122CC26CA2A844EC66B
:1034400006CE4AC8AE84EFD04F888947744C7CCCF6
:103450003C4C0547AA8985073CCC6395E6061C547D
:1034600081C77370043001A097D701009387870C40
:103470009C43ADE7130944004A85EFD06F8F97D77F
:1034800001009387E70C48549C4363F6A70097D745
:10349000010023AFA70AD145EF30C03997D701000B
:1034A0009387071ECA853E95EFD00F8897D70100F6
:1034B0009387870B9C435854DC5763F5E70099C00A
:1034C00085479CC06244F240D24442494E85B2498D
:1034D00005616FC03FFF7370043001A09305840144
:1034E00017D501001305C528EFD00F84C1B7AA87EF
:1034F00029C57370043017D701001307270514433B
:103500009DE2F04F894601456315D60023AE0704BE
:1035100005451C4381CB97D701009387E704984367
:10352000784315E3828097D601009386E6039042A4
:1035300094427442850674C2E9B797D70100938715
:10354000A7029C437DB7984394437C43FD177CC3FB
:10355000FC42E9FB7360043082805D71A6C24EDEDE
:1035600052DC56DA5AD85ED686C6A2C4CAC062D425
:1035700066D26AD097D901009389090017DB010050
:10358000130BCBFE97D40100938484FE97DA0100DD
:10359000938A4AFE054AA54B83A709009843630B0B
:1035A0000712DC4703A90700EFE06FF6EFE02FF703
:1035B00083270B002A8C6369F50A97D7010023A79C
:1035C000A7FA0146637B251B8840B3058941EFD0EC
:1035D000DFBDEFE0DF98630B0512884081460146AE
:1035E0008A85EFD0EFEB4DD98247224463DA07009A
:1035F0009247B245228582978247E3C007FE224464
:103600005C4889C713054400EFC09FF6EFE02FF137
:1036100083270B002A8C6360F50A824717D70100C5
:10362000232687F5E3EBFBFAB317FA0013F707211C
:10363000631F072013F7770C6314071C93F7070227
:10364000C9DF2285EF00301A49BFDC47C04783AC91
:103650000700130944004A85EFC09FF15C502285A2
:1036600082975C4C6387470B83A70900984371FFDF
:1036700003A70A0097D6010023AA86EF97D6010078
:1036800023AAF6EE97D7010023A8E7EEEFE03F8DDF
:10369000A9B7DC4703A9C70003AD0700930C490095
:1036A0006685EFC0FFEC832749024A85829783270E
:1036B000C9016386470983A70900984379FB03A7DB
:1036C0000A0097D6010023A7F6EA97D7010023A5A1
:1036D000E7EAA1B7EFE0AFE3EFE06FE483270B0089
:1036E0002A8CE363F5F883A70A00884001499043D8
:1036F000B305894117D70100232A87E7133616003F
:10370000EFD0BFAAEFE0BF85E31905ECEFC01FD0F3
:10371000E9B51C4CCA85E69763EAFC049C4089CF56
:1037200002C866CA22CCEFF0CFE688408146014647
:103730000C08EFD0CF860DF97370043001A08327F9
:103740008901E685EA97636CFD049C4089CF02C835
:103750006ACA4ACCEFF0EFE38840814601460C0884
:10376000EFD0EF8329F97370043001A003A509009D
:103770005CC000C8EFC0DFDCC5BDEFE04FFE83A733
:103780000900DC47C047930C44006685EFC05FDE4C
:103790005C4C638F47015C50228582973DBD03A539
:1037A00009002322F90023282901EFC07FD921B77E
:1037B0001C4C00C83307F90058C0636DEC02330C91
:1037C0002C416363FC029C4089CF02C84ACA22CCC8
:1037D000EFF02FDC8840814601460C08EFC03FFC2B
:1037E0005DF97370043001A003A50A00E685EFC0FF
:1037F0003FD555B703A50900E685EFC07FD461BF6B
:103800009247144C00C83387D70058C0636FEC064A
:10381000B307FC4063E4D7065C50228582975C4C7A
:10382000E39D47DB144C92479840B69711CF02C8EE
:103830003ECA22CCEFF0EFD58840814601460C0805
:10384000EFC0FFF5E31B05D87370043001A0924769
:103850001CCC95C3E2975CC000C893054400636725
:10386000FC0003A50A00EFC0BFCD85BB03A509007E
:10387000EFC01FCD9DB37370043001A003A50A00F3
:1038800093054400EFC0DFCB89BB6374FC00E37594
:10389000F7F803A5090093054400EFC07FCA35BBC4
:1038A000411122C406C626C24AC017D4010013041F
:1038B00024CCEFF0CFE21C4095CBEFF08FE41C401E
:1038C0009DC381480148814709478146130600404E
:1038D00097D50100938585AE17050000130525C80F
:1038E000EFD0DF9939E97370043001A017D90100D6
:1038F0001309C9EB4A85EFC09FC197D40100938497
:1039000024EC2685EFC0BFC00146C145114597D7BD
:10391000010023A327C797D7010023AD97C4EFC0A9
:10392000FFDA17D701002325A7C411CD97D50100D1
:10393000938545A8EFD02FFC49B7B240224492446A
:103940000249410182807370043001A0A5C97971D8
:1039500056CAAA8A1305C00222D426D24AD04ECE15
:1039600052CC06D65AC85EC63A89B689328AAE8427
:10397000912B2A8405C9EFF08FD697D70100938742
:1039800027BF9C439DCFEFF0CFD7130544002320E2
:10399000540104CC232E4401232034032322240386
:1039A000EFC03FB82285B250225492540259F249D6
:1039B000624AD24A424BB24B4561828073700430F6
:1039C00001A097DB0100938B6BDE5E85EFC03FB4F7
:1039D00017DB0100130BCBDE5A85EFC05FB3014646
:1039E000C145114597D7010023A877B997D70100A2
:1039F00023A267B9EFC09FCD17D70100232AA7B62E
:103A000001C997D501009385E59AEFD0CFEEA5BF08
:103A10007370043001A039C5011122CC06CE26CA2C
:103A200017D401001304C4B4832804002A88014574
:103A300063850802BA842EC0368732C242C49546D6
:103A400063C5B602EFF0EFB48947630BF502084097
:103A5000814601468A85EFC09FD4F2406244D24439
:103A6000056182807370043001A08A8581463A86A0
:103A70004685EFD00F88F2406244D24405618280CF
:103A80000840814626868A85EFC07FD1F9B719C1E3
:103A9000084182807370043001A001E57370043026
:103AA00001A0411106C622C42A84EFF04FC3484842
:103AB0003334A000EFF0EFC42285B240224441012C
:103AC000828001E57370043001A0411122C42A8470
:103AD00006C6EFF0CFC00050EFF0AFC2B240228573
:103AE00022444101828001E57370043001A041113C
:103AF00022C426C22E84AA8406C6EFF04FBE80D010
:103B00002244B240924441016FF0AFBF011106CE92
:103B100097D701009387C7A52AC28843B6872EC4CA
:103B200032C68A853E868146F9573EC0EFC07FFC8B
:103B3000F2400561828097D70100938767A383A82D
:103B40000700639508007370043001A00111B2876B
:103B50002E872A8836868A8546858146FD5806CE78
:103B600046C042C23AC43EC6EFC07FC3F2400561C0
:103B7000828001C9B70700FFED8F99C773700430C9
:103B800001A07370043001A0411122C426C206C6F0
:103B90002A84AE84EFF0AFB4184093C7F4FFF98FD6
:103BA0001CC02244B240924441016FF08FB509C954
:103BB000370700FFB3F7E50099C77370043001A021
:103BC0007370043001A06F20705C4111714522C4F4
:103BD00006C6CD2C2A8411C5232005001105EFC08F
:103BE0001F932285B24022444101828001CDB70754
:103BF00000FFED8F81C77370043001A099E57370E9
:103C0000043001A07370043001A0011122CC4AC815
:103C10004EC652C456C206CE26CABA893689B28A60
:103C20002E842A8AEFF0EF9611E563850900737000
:103C3000043001A0EFE0AF8D83240A00B377940035
:103C40006316090295C763870A009347F4FFE58F5F
:103C50002320FA00EFE0AFB0F240624426854249EB
:103C6000D244B249224A924A05618280E30DF4FCB3
:103C7000E38209FEB3355001E20563050900B70789
:103C80000004DD8D4E86C18D13054A00EFE09FDAFA
:103C9000EFE0EFAC19E1EFC06FF7EFF06FA993170A
:103CA0006500AA8963D80700B7040001FD14B3F4C6
:103CB00099005DB7EFF0AFA283290A00B377340112
:103CC000631E090089CB63880A009347F4FFB3F7AA
:103CD00037012320FA00EFF0CFA2F9B7E31DF4FE7D
:103CE000DDB701C9B70700FFED8F99C773700430C6
:103CF00001A07370043001A0411122C42A8406C6B9
:103D000026C24AC02E89EFF08F9D04409345F9FFEB
:103D1000B3F795001CC0EFF0CF9EB2402244268539
:103D200002499244410182802E868146AA85170568
:103D30000000130545E46FF07FDD411122C42A84A1
:103D400006C6EFC08FF80040EFC0CFF7B240228523
:103D500022444101828009C9370700FFB3F7E5001B
:103D600099C77370043001A07370043001A06F20F4
:103D7000F041B70700FFF18F81C77370043001A0D5
:103D800001E67370043001A0011122CC4AC84EC66E
:103D900052C406CE26CA3689AE892A8A3284EFE01A
:103DA0005FFF21E1630509007370043001A0EFD0CB
:103DB0001FF683240A00CE855285B3E49900613F43
:103DC000B37794006307F40683240A00EFE02F9989
:103DD000F240624426854249D244B249224A0561F2
:103DE0008280EFD0DFF283240A00CE855285B3E4CF
:103DF00034019537B3F78400638D8702E30609FC2D
:103E0000B70500054A86C18D13054A00EFE09FC241
:103E1000EFE0EF9419E1EFC06FDFEFF06F919317D0
:103E20006500AA8463DF0700B7070001FD17FD8C5A
:103E300045B783270A001344F4FFE18F2320FA00DB
:103E400071B7EFF0CF8983240A00B37794006397AA
:103E500087009347F4FFE58F2320FA00EFF06F8A85
:103E6000E1B7411122C406C62A8426C2EFD03FEA38
:103E70005C4085C308489304C4006316950015A0F0
:103E8000084863009502B7050002EFE0BFD75C4029
:103E9000E5FB2285892A2244B240924441016FE029
:103EA0000F8C7370043001A0B2862E86AA85170588
:103EB0000000130505D06FF07FC519C1084D828041
:103EC00001458280411122C406C62A84EFD03FE416
:103ED00097C701009387876A9C43A1EBE56717D7D3
:103EE00001001307678FF11797C6010023AEE6683C
:103EF00017C701002328F76817D701002320F78E82
:103F000097C701009387C76717D701002326F78C4F
:103F1000854717C70100232B076617C70100232118
:103F2000076617C70100232BF76419E8EFE02F831A
:103F3000EF10600801442285B24022444101828092
:103F40001305840093773500C1EFE5671307F5FF8C
:103F5000E917E3EDE7FC97C601009386E6629C4211
:103F600029A0984311C7BE86BA87D843E36BA7FE42
:103F700017C701001307C760E38AE7FA9843414671
:103F80001384870098C2D843B306A7406378D6024B
:103F90003388A7002322D800C8C38325480097C6CA
:103FA00001009386665E11A0BA8698425043E36D85
:103FB000B6FE2320E80023A00601D84397C70100DE
:103FC0009387C7609C43998F17C701002320F76030
:103FD000EFD0FFF831DC2285B240224441018280DB
:103FE000719911059DB729C9411122C406C62A84B9
:103FF000EFD0FFD1930584FF0326C4FF17C701004C
:104000001307875811A03E871C43D443E3EDC6FE37
:10401000232CF4FE0CC397C701009387275B9843BA
:104020008327C4FF2244B240BA9717C70100232F49
:10403000F75841016FD0BFF2828097C70100938784
:10404000E7588843828082803367B5000D8BAA874A
:104050001DE79308D6FFAA982A87AE8663711503D9
:1040600003A8060011079106232E07FFE36A17FF36
:104070009347F5FFC697F19B9107BE95AA972A969D
:1040800063F3C70A9386450013884700B3B6D70089
:1040900033B8050133E7F50093C61600134818003E
:1040A0000D8BB3E6060113371700758F330EF640FC
:1040B0009386170029CF1337AE0031EB13532E0030
:1040C0002E88BE860147832808000507110823A013
:1040D00016019106E36967FE1377CEFFBA95BA978A
:1040E0006302EE0483C60500138717002380D70000
:1040F000637AC70283C6150013872700A380D70001
:104100006372C70203C725002381E7008280B307DB
:10411000F640AE97850503C7F5FF8506238FE6FEBB
:10412000E39AF5FE82808280B367C5008D8BB30869
:10413000C500E9C36371150FB307A0408D8B1387CA
:104140003700954693F5F50F130815003383A84003
:104150007D166373D70015476363E60CD5CF230044
:10416000B5000547638DE700A300B5000D471308B0
:1041700025006396E700130835002301B500139668
:1041800085004D8E13970501518F3303F3409396AD
:104190008501D98E13562300AA97014794C30507BA
:1041A0009107E36DC7FE1377C3FFB307E80063070A
:1041B000E3062380B70013871700637C1703A380EF
:1041C000B70013872700637617032381B70013878F
:1041D000370063701703A381B70013874700637A22
:1041E00017012382B7001387570063741701A38256
:1041F000B700828093F5F50F13978500D98D13973B
:1042000005014D8FE37715FFAA87910723AEE7FEDF
:10421000E3ED17FF828082802A8895B78280AA8783
:1042200049BF834705002A8799C7050583470500CD
:10423000EDFF198D82800145828005058347F5FFDA
:10424000850503C7F5FF91C7E389E7FE3385E7409E
:1042500082808147E5BFAA87850503C7F5FF8507EB
:10426000A38FE7FE75FB828083460500930700025B
:104270006397F600050583460500E38DF6FE9387F8
:1042800056FD93F7D70F85C7AA87814585CE01458F
:104290008507138606FD1317250083C607003A9588
:1042A00006053295F5F699C13305A04082809385C5
:1042B00036FD8346150093B5150093071500E1FA06
:1042C0000145D5B7014582809C412380A7009C41D0
:1042D00085079CC1828097C601009386662B9C420D
:1042E000175703001307075213861700BA97238046
:1042F000A70097C5010023ADC528A9476308F500AD
:10430000930700046305F6000145828075DE3706D9
:1043100010F005078347F7FF2320F6F09C42FD17B6
:1043200097C5010023A6F526EDF7014582804D7162
:104330002322911423202115232A5113232481138E
:104340002326111423248114232E3113232C4113EB
:104350002328611323267113232291132320A113F1
:10436000232EB111AA842E8932C6130C5002A54AFD
:104370008347090063808703B9CB804011A0A1CB9C
:104380002300F40080400509050480C0834709002C
:10439000E39787FF0346190093081900C686130D9B
:1043A0000002FD597D5A0148130550059307D6FDBB
:1043B00093F7F70F138916006363F52A17C70100F7
:1043C000130747C48A07BA979C43BA97828783200A
:1043D000C114032481148324411403290114832963
:1043E000C113032A8113832A4113032B0113832B47
:1043F000C112032C8112832C4112032D0112832D33
:10440000C11171618280A14C02C4854763D5071533
:10441000B2478040938B770093F68BFF03AB060087
:1044200083A94600938786003EC6668681465A85E4
:10443000CE85EF1030702AC8814763853723930DEE
:104440004101854B668681465A85CE85EF10D01096
:10445000814666862A8BAE89EF10D06DA24723A0D5
:10446000AD0093861B00910D63843701B68BD9BFD5
:10447000E37E9BFF63DD4601A2872380A701804086
:104480007D1A930714009CC03E84E3C846FF9396B0
:104490002B001C08BE9631A8938777052300F400F3
:1044A0008040FD1B93871B00050480C0F116E3517B
:1044B000F0EC9C42E3E2FAFE93870703C5B79C4009
:1044C0009306000332472380D7009C4093064700A1
:1044D000C14C1386170090C013068007A380C70045
:1044E000804002C4BA87050480C003AB070081493D
:1044F00036C625BFB24783AC0700938B4700638461
:104500000C1C635F40199307D0026319FD1683C723
:104510000C0085C363DC09189440850C7D1A238048
:10452000F6008040050480C083C70C00E5F7635D9A
:1045300040018040930700022300F40080407D1A70
:10454000050480C0E31A0AFE5EC61DB502C4854795
:10455000A94CE3CF07EBB24780409386470071B781
:1045600003C61600CA8699B59C4093065002238064
:10457000D7008040050480C0E5BBC14C02C471B5C2
:10458000B24703C61600CA8683A9070091073EC634
:10459000E35E0AE04E8AFD5911BD03C61600130DF5
:1045A000D002CA8621B59347FAFFFD8703C61600DD
:1045B000337AFA00CA86DDBB03C61600130D00036A
:1045C000CA86EDB383C51600930906FDCA86938794
:1045D00005FD2E86E3EEFAFA93972900BE9985062B
:1045E0008609AE9983C50600938909FD938705FD69
:1045F0002E86E3F3FAFE69BF32479C40144311074D
:104600003AC62380D7008040050480C095B3854713
:1046100063D3070BB24793867700E19A93878600AE
:104620003EC683A946009C4263DC090A94401306F7
:10463000D002B307F0402380C6008040B336F000BC
:10464000B3093041050480C03E8BB389D940A94CE1
:1046500002C4E1BB03C616000508CA8681BB9C40A4
:10466000468921B7E37D9BDD8547814B8546E3C5C0
:1046700047E131BD97CC0100938CCCD4CE856685C3
:10468000EF10C015330AAA40635C4001804023004C
:10469000A40180407D1A050480C0E31A0AFE014A85
:1046A00083C70C00E38207EAE3C809E6FD197D57DA
:1046B000E394E9E6ADBDB247938647009C4336C616
:1046C00093D9F74195B7635640019307D002E3139E
:1046D000FDFA97CC0100938CECCE930780021DBDB0
:1046E0003E8BA94C02C4804089B34D71232E3113F7
:1046F000B70900409387F9FF2324811423229114E2
:10470000232C4113232A511323261114232021156E
:104710002328611323267113232481132322911349
:104720002320A113232EB1112A8A2EC417C40100FD
:10473000130404E6975A0300938ACA0C97C4010035
:104740009384C4A13EC69305500229451308000472
:10475000B70610F083470A006386B704C1C7184044
:10476000050A13061700569797C8010023A2C8E24E
:104770002300F7006382A706E31E06FD1757030018
:104780001307470805078347F7FF23A0F6F01C40EF
:10479000FD1717C60100232DF6DEEDF783470A004B
:1047A000E39EB7FA83461A0013051A002A87930B73
:1047B00000027D5B7D5C014893055005A548938709
:1047C000D6FD93F7F70F130A170063E7F5348A074E
:1047D000A6979C43A6978287175703001307870263
:1047E00055F28DBF8320C114032481148324411406
:1047F000032901148329C113032A8113832A411336
:10480000032B0113832BC112032C8112832C411221
:10481000032D0112832DC11171618280A14C014DC4
:10482000854763DB0719A2479D07E19B83AD07001E
:1048300003AB4700138787003AC4668681466E85BE
:10484000DA85EF10302F2AC863066D351309410150
:104850008549668681466E85DA85EF10E04F66866B
:104860008146AA8D2E8BEF10F02C2320A9008509FC
:104870001109E3106DFFE3FE9DFD13060004B7066A
:1048800010F063D189031C4013871700D69797C592
:10489000010023AFE5CE23807701630CC7047D1CA4
:1048A000E3C389FFB2476800A548B386F9008A06CA
:1048B0001C08BE96294813030004370610F0E38451
:1048C000A6E89C429305000363F4F8009305700585
:1048D0001840AE9793051700569717CE010023296D
:1048E000BECA2300F7006380072B638C6526F11690
:1048F000F9B7175703001307E7F005078347F7FFDA
:1049000023A0F6F01C40FD1797C5010023A2F5C8AF
:10491000EDF77D1C71B71C401306000413871700C8
:1049200097C5010023A6E5C6B386FA0093050003E8
:104930002380B6006300C73E890797C6010023A9FC
:10494000F6C45697930680072300D7001757030035
:10495000130747EBB70610F0639EC70005078347B0
:10496000F7FF23A0F6F01C40FD1717C60100232116
:10497000F6C2EDF7A247C14C014D91072247014B0A
:10498000832D07003EC455BDA24783AC07001389A1
:104990004700638F0C3A635480219307D002639ED3
:1049A000FB2E03C70C00BA856310072025AC854792
:1049B000A94C014DE3C907E7A2479107C1B7A24738
:1049C00083461700528703AB070091073EC4E358A4
:1049D0000CDE5A8C7D5BE5B383461700930BD00247
:1049E0005287F1BB9347FCFFFD8783461700337C5A
:1049F000FC005287E9B383461700930B00035287EC
:104A00007DBB03461700138B06FD5287930706FDF7
:104A1000B286E3EEF8FA93172B00DA9705078607BC
:104A2000B29703460700138B07FD930706FDB28676
:104A3000E3F3F8FE69BFA2451C40294698419386DE
:104A40001700D69717C501002324D5B42380E700AB
:104A5000138945006301C72A930700046387F62082
:104A60004AC4D5B1854763DF0729A247138777007A
:104A7000619B930787003EC4032B47001C43635B85
:104A80000B301840130600049306170097C5010069
:104A900023A0D5B056979305D0022300B7006388B2
:104AA000C62CB307F0403337F000330B6041BE8DA6
:104AB000330BEB40A94C014D49B383461700050861
:104AC0005287F5B9834617005287D5B91C40930623
:104AD00000041387170017C60100232BE6AAD697F8
:104AE000130650022380C700E31FD7C417570300E3
:104AF000130747D1B70610F005078347F7FF23A038
:104B0000F6F01C40FD1717C601002323F6A8EDF7A9
:104B10001DB9C14C014D29B31C40930600042A8ADB
:104B20001387170017C601002324E6A6D69713069D
:104B300050022380C700E318D7C01757030013079C
:104B400067CCB70610F005078347F7FF23A0F6F000
:104B50001C40FD1717C60100232CF6A2EDF72A8A88
:104B6000DDB6175703001307E7C905078347F7FFAB
:104B70002320F6F01C40FD1797C5010023AAF5A0DD
:104B8000EDF7F1162DBB175703001307A7C7F1FD6B
:104B9000F11635B3E3FC9DCB8549C5B1014C03C784
:104BA0000C00BA85E30E07EAFD58294513080004F6
:104BB000B70610F063570B0A1C4013861700D697F0
:104BC00017C301002326C39C2380E7006384A50646
:104BD00063040609850C03C70C007D1CBA8579FBAC
:104BE000E35080E91C409305000213060004B70659
:104BF00010F021A07D1CE3050CE613871700D69763
:104C00002380B70017C501002324E598BA87E31372
:104C1000C7FE175703001307E7BE05078347F7FFD3
:104C200023A0F6F01C40FD1717C501002322F596BE
:104C3000EDF7C9B7175703001307C7BC41DE0507D7
:104C40008347F7FF23A0F6F01C40FD1717C60100AD
:104C50002320F694EDF7BDBF17570300130787BA5B
:104C6000F9BF7D1BE31A1BF5A5BF175703001307F8
:104C700067B9B70610F005078347F7FF23A0F6F0E2
:104C80001C40FD1717C601002324F690EDF74AC417
:104C90005DBC97BC0100938CEC72DA856685EF00F1
:104CA000F033330CAC40E35C80EF1C40130600048F
:104CB000B70610F021A07D1CE3020CEE138717004D
:104CC000D6972380770197C5010023A3E58CBA8787
:104CD000E313C7FE175703001307C7B2050783473F
:104CE000F7FF23A0F6F01C40FD1797C5010023A194
:104CF000F58AEDF7C9B7175703001307A7B0B5FA40
:104D00004AC491B4A247138747009C433AC413DBBB
:104D1000F741B5B3175703001307C7AEB70610F036
:104D200005078347F7FF23A0F6F01C40FD1717C6C1
:104D30000100232FF684EDF7854717C701002329CB
:104D4000F7849307800717570300230DF7AA1DB1B7
:104D5000635680019307D002E39DFBF297BC0100EC
:104D6000938C4C66130780029305800235BD9756DD
:104D70000300938626A9370610F0850603C7F6FFC1
:104D80002320E6F018407D1797C5010023A2E58097
:104D90006DF701BBBE8DA94C014D45B4B70710F0AE
:104DA00023A0A7F201A03971130341022ED29A85E4
:104DB00006CE32D436D63AD83EDA42DC46DE1AC6C1
:104DC0002D32F2400145216182805D711303810320
:104DD00022D42AC632DC2A841A86680006D6BEC2CD
:104DE00036DEBAC0C2C4C6C61ACEEFF04FD4B24740
:104DF000238007003245B250018D225461618280C8
:104E0000B70710F083A647F403A607F403A747F4F7
:104E1000E31AD7FE8566938606FAB29633B6C600C5
:104E2000B305E60023A4D7F423A6B7F48280B7071E
:104E300010F003A747F403A607F483A647F4E31A88
:104E4000D7FE8566938606FAB29633B6C60023A4CB
:104E5000D7F4B305E60023A6B7F49307000873A0C0
:104E600047308280411122C406C651447D14EF00B0
:104E700050016DFCB240224441018280411122C4A4
:104E800006C697B701009387277117B40100130472
:104E9000647098431C401306F07C93064706938782
:104EA000470697B5010023A9D56E97B5010023A346
:104EB000F56E6346D600B24022444101828013075A
:104EC000478997B7010023A9E76CEF009009854750
:104ED0006310F502184085679387F7760145E3DC98
:104EE000E7FCEFF0BFEB2244B24041016FC03FE16D
:104EF00017B501001305854DEFF0FFEA0945EFF006
:104F0000FFE92244B24041016FC07FDF17B50100C5
:104F10001305454D6FF03FE917B501001305054D29
:104F20006FF07FE8411122C426C206C6856417B41B
:104F300001001304244C938784380100FD17F5FF0A
:104F40002285EFF05FE6C5BF411106C622C4EF001F
:104F5000006717070000130727F1814605469305F0
:104F6000200317B5010013056549EFE03F9E2A8431
:104F7000EFC0FFDA2A8622852244B24001478146EB
:104F8000854541016FE03FA9411106C6EF00607DF4
:104F9000054781476316E500B2403E8541018280A6
:104FA00017B5010013058542EFF0FFDFB2408947D6
:104FB0003E85410182807370043001A0828073704D
:104FC000043001A0411126C24AC006C622C42A8963
:104FD000EFD07FDB97B701009387C75D9C43954473
:104FE0006387A70617B401001304445D0145EFD0A1
:104FF000FF8208407D5781460546A685EFE01FBF2A
:1050000075F525A0EFD09F810840FD563D46CA8525
:10501000EFE03FD63D897D5785460146BD45631D7E
:1050200095020840EFE09FBC0DE50145EFD00FFF72
:105030000840FD563D46CA85EFE0BFD39374F500A6
:10504000BD470145E380F4FC7370043001A08D443A
:1050500051BF7370043001A07370043001A00111BE
:1050600022CC4EC652C406CE26CA4AC817B4010086
:105070001304C45497B901009389C954130AF00F5B
:105080000145EFD0AFF908407D5785460546894573
:10509000EFE0DFB52A8908407D5785460146930534
:1050A000200AEFE0BFB41375250A9307200A854450
:1050B0006304F50C0145EFD06FF608407D57854637
:1050C00005469305200AEFE07FB26303450185445E
:1050D0000145EFD0AFF40840FD563D468945EFE06D
:1050E0005FC93D89BD476303F5008544084081459C
:1050F000EFE07FC625C5084081458544EFE07FBECF
:105100000145EFD0AFF10840FD563D468945EFE03F
:105110005FC63D89BD476303F5008544084081456E
:10512000EFE07FC319C908407D5785460146BD455C
:10513000EFE0DFAB7370043001A008407D57854677
:105140000146BD45EFE09FAA75F5EDF483A7090080
:10515000850717B701002327F7461DB7084081458B
:10516000EFE03FB819ED91EC83A70900850717B769
:1051700001002329F74469B79304E9F5B33490009B
:1051800015BF8544B5BF79714AD006D622D426D240
:105190004ECE52CC56CA5AC85EC662C466C26AC0F7
:1051A0002A89EFE09FA297B7010023A9A7406300D7
:1051B000054017BA0100130AEA3F03250A0097B910
:1051C00001009389E93E0544EFC0CFD1AA8403A52D
:1051D0000900EFC02FD18D47630EF53CA14B854AE6
:1051E00097B401009384843D094B0D4C03250A00BC
:1051F000EFC0EFF303A50900EFC06FF303250A002A
:10520000EFC04FCE63036501054403A50900EFC05D
:105210006FCD6303650105448840D685EFE0BFB3D9
:1052200093F73A0003250A0063950734EFC08FCB4C
:1052300063036501054493F75A0003A509006395CC
:105240000732EFC02FCA630365010544FD1B860AC0
:10525000E39E0BF803250A0017BD0100130DCD36A0
:10526000894AEFC0CFEC03A50900854B930C000AD7
:10527000EFC0EFEB88400D4B130CD005EFE07FBE85
:10528000EFE0BF9497B7010023AAA732630E053061
:105290004A85EFC0CFE94A85EFC0CFC4630355010B
:1052A000054488409305200AEFE0FFAA88400147A3
:1052B000814601469305F00FEFE05F93630395018C
:1052C00005444A85EFC00FC2630355010544884079
:1052D0009305D00FEFE03FA8884001478146014683
:1052E0009305F00FEFE09F909307D00F6303F50055
:1052F00005444A85EFC00FBF63035501054488404C
:105300008945EFE05FA54A85EFC0CFBD6303650126
:10531000054488408145EFE01FA49307F00F630325
:10532000F500054488408945EFE0BF9B9307F00FE7
:105330006303F50005444A85EFC06FDF4A85EFC07F
:105340006FBA63035501054488408945EFE0BFA06B
:105350004A85EFC02FB963036501054488400147C2
:10536000814601469305F00FEFE05F8863038501F6
:10537000054488409305F00FEFE0BF966303850175
:10538000054488408145EFE0DF9511C105444A8519
:10539000EFC04FB563036501054403250A00EFC064
:1053A0006FB463036501054403A50900EFC08FB323
:1053B0006303650105448840B945EFE0DF99884003
:1053C000FD5605468545EFE0DF9A058911E1054464
:1053D00088408145EFE0FF90B9476303F50005443D
:1053E0008840B945EFE0FF8F88408145EFE07F8F2F
:1053F00011C105444A85EFC08FD303250A00EFC0D1
:105400000FD303A50900EFC08FD24A85EFC08FAD3F
:1054100063035501054403250A00EFC0AFAC6303E5
:105420005501054403A50900EFC0CFAB6303550147
:1054300005448840FD563D468545EFE09F933D89F4
:10544000BD476303F500054488408145EFE07F894F
:1054500011C105444A85EFC0EFA863036501054407
:1054600003250A00EFC00FA863036501054403A5E7
:105470000900EFC02FA76303650105444A85EFC00B
:105480000FCB03250A00EFC08FCA03A50900EFC0A8
:105490000FCA4A85EFC00FA56303550105440325D4
:1054A0000A00EFC02FA463035501054403A50900BA
:1054B000EFC04FA363035501054489450145EFC083
:1054C0000FB58840FD563D468545EFE09F8A3D89F2
:1054D000BD476303F500054488408145EFE07F80C8
:1054E00011C105444A85EFC0EF9F63037501054470
:1054F00003250A00EFC00F9F63037501054403A550
:105500000900EFC02F9E63037501054401458145E5
:10551000EFC0EFAF4A85EFC0EF9C63035501054430
:1055200003250A00EFC00F9C63035501054403A542
:105530000900EFC02F9B6303550105448840EFE04D
:105540005F924A85EFC00F9A630365010544032506
:105550000A00EFC02F996303650303A50900EFC09C
:105560006F987370043001A0EFC0CF97E31F85CD13
:10557000F1B9EFC02F97E31F85CB75B903A50900DB
:10558000EFC04F96E31F65FD69FC83270D0085077B
:1055900017B70100232AF702EFE02FE397B70100C6
:1055A00023AEA700E31605CE7370043001A073701C
:1055B000043001A01384D4FF3334800005B10111FD
:1055C000814801487C00054781461306004097B595
:1055D00001009385E5E317050000130585A806CEB5
:1055E000EFB0DFC9B2468148014881470147130641
:1055F000004097B50100938525E2170500001305CB
:10560000C5B8EFB0BFC78148014897B7010093877D
:1056100067FA054791461306004097B50100938548
:1056200025E0170500001305259AEFB03FC597B791
:1056300001009387E7F7814801480547A146130613
:10564000004097B501009385A5DD170500001305FF
:10565000A597EFB0BFC297B70100938767F59C434A
:1056600099CBEFE08FD697B7010023A7A7F419C510
:10567000F240056182807370043001A073700430C1
:1056800001A0411106C622C497B70100938707F213
:105690009C4313074006850797B6010023A8F6F040
:1056A000638EE7001307800C6388E7061307C012B8
:1056B0006387E702B24022444101828017B40100AF
:1056C000130484EF0840EFE04FE715CD854717B787
:1056D0000100232BF7ECB24022444101828097B7AE
:1056E0000100938767ED8843C945EFE0EFE3854705
:1056F0006304F50417B701002328F7EA97B7010000
:1057000023A607EA45BF08400146C945EFE0CFF9A7
:105710008547E31DF5FA79BF97B701009387C7E97D
:105720008843EFE08FE1C947E306F5F8854717B7EF
:105730000100232BF7E645B797B701009387C7E62B
:105740009C4317B70100232307E6ADF797B7010085
:10575000938707E79C43850717B701002322F7E6E5
:1057600091BF17B70100130727E68328070097B7F3
:105770000100938727E50C4317B60100130646E2A4
:105780009443104217B801001308C8E1032708002A
:1057900017B501002328B5E001456306D60033079D
:1057A00017413335E000904317B70100130747E175
:1057B00097B70100938787DE14439C43184397B53E
:1057C000010023AFC5DC958FB337F000B307F0407D
:1057D00097B6010023A4E6DC7D8D8280B305B50079
:1057E000930705006386B70003C707006316070029
:1057F0003385A74067800000938717006FF09FFEF6
:10580000130101FB23229104232C41032322910342
:10581000232611042324810423202105232E310370
:10582000232A5103232861032326710323248103A0
:105830002320A103232EB101930C0500138A050038
:105840009304000063DE05003305A0403337A00059
:10585000B305B040930C0500338AE5409304F0FF94
:1058600063DA06003306C040B337C000B306D04049
:10587000B386F640930A06009389060013840C0051
:1058800013090A006396062817BB0100130B8BA2AD
:105890006370CA16B70701006372F6149307F00F1E
:1058A00063F4C70093098000B3573601330BFB0044
:1058B00083470B0013050002B3873701B309F54096
:1058C000638C0900B3153A01B3D7FC00B31A360153
:1058D00033E9B70033943C0113DB0A0193050B0055
:1058E00013050900EF00507C130A050093050B0017
:1058F000939B0A0113050900EF00907693DB0B01DF
:105900009305050013850B00EF00D072131A0A01EE
:1059100093570401B367FA0063FAA700B3875701EE
:1059200063E6570163F4A700B38757013389A740A3
:1059300093050B0013050900EF001077130A05000B
:1059400093050B0013050900EF0090711314040177
:1059500093050500131A0A0113850B001354040163
:10596000EF00506D33648A00637AA400330454015D
:10597000636654016374A400330454013304A440E7
:105980003354340193050000638A040033048040DB
:10599000B3378000B305B040B385F540130504006C
:1059A0008320C104032481048324410403290104C6
:1059B0008329C103032A8103832A4103032B0103A3
:1059C000832BC102032C8102832C4102032D01028F
:1059D000832DC1011301010567800000B707000195
:1059E00093090001E362F6EC930980016FF0DFEBAD
:1059F000631A06009305000013051000EF005066BF
:105A0000930A0500B707010063FAFA0E9307F00F37
:105A100063F4570193098000B3D73A01330BFB00BD
:105A200083470B001305000233095A41B38737013E
:105A3000B309F540E38209EAB39A3A01335BFA000D
:105A4000B3153A01B3D7FC0093DB0A0133E9B70081
:105A500013050B0093850B00EF001065130A05007A
:105A600093850B00139C0A0113050B00EF00505F98
:105A7000135C0C019305050013050C00EF00905B0F
:105A8000131A0A0193570901B367FA0033943C01D2
:105A900063FAA700B387570163E6570163F4A700D1
:105AA000B3875701338BA74093850B0013050B0079
:105AB000EF00905F130A050093850B0013050B00A0
:105AC000EF00105A9305050013050C00EF009056E7
:105AD00093160901131A0A0193D60601B366DA0078
:105AE00063FAA600B386560163E6560163F4A60086
:105AF000B38656013389A6406FF01FDEB707000159
:105B000093090001E3EAFAF0930980016FF0DFF0F6
:105B10006376DA0093050A006FF01FE7B70701000C
:105B200063FAF604930BF00F33B5DB001315350061
:105B300033D7A60097A701009387C777B387E700FD
:105B400083CB070093050002B38BAB00338B754109
:105B5000631C0B0263E4460163EACC003384CC404F
:105B6000B306DA4033B98C00338926419305090026
:105B70006FF09FE1B707000113050001E3EAF6FAB1
:105B8000130580016FF0DFFAB3966601335D76018D
:105B9000336DDD00B35D7A01B3156A0133DC7C013E
:105BA00013540D01336CBC0013850D0093050400E4
:105BB000B3196601EF00504F930A050093050400E6
:105BC00013850D0033996C01931C0D01EF005049B2
:105BD00093DC0C01130A05009305050013850C00E6
:105BE000EF005045939A0A0113570C0133E7EA007E
:105BF000930D0A00637EA7003307A701930DFAFFF8
:105C00006368A7016376A700930DEAFF3307A70136
:105C1000330AA7409305040013050A00EF00D0489B
:105C200093050400930A050013050A00EF00504392
:105C3000930505001304050013850C00EF00903F49
:105C400093150C01939A0A0193D50501B3E5BA00A7
:105C50001307040063FEA500B385A5011307F4FF35
:105C600063E8A50163F6A5001307E4FFB385A5016A
:105C7000939D0D01B70C0100B3EDED001384FCFF03
:105C8000B3F78D0033F48900338AA54013850700EC
:105C9000930504002326F10093DD0D01EF009039F8
:105CA00093050400930A050013850D00EF0090385A
:105CB00013DC090193050C002324A10013850D00BA
:105CC000EF0050378327C10013040C009305040034
:105CD000130C050013850700EF00D03583268100E3
:105CE00013D70A013305D5003307A7006374D70023
:105CF000330C9C01B70701009387F7FF9355070109
:105D00003377F70013170701B3F7FA00B38585015E
:105D1000B307F7006366BA00631EBA00637CF9003C
:105D200033863741B3B7C700B385A541B385F54086
:105D300093070600B307F9403339F900B305BA40B9
:105D4000B385254133947501B3D767013364F400FB
:105D5000B3D565016FF05FC3130101FD23229102EA
:105D6000232A510123261102232481022320210307
:105D7000232E3101232C41012328610123267101A7
:105D800023248101232291012320A101930A0500EC
:105D900093840500639E06381304060093090500EA
:105DA00017A901001309095163F8C512B7070100CB
:105DB000138B05006378F6101307F00F3337C70015
:105DC00013173700B357E6003309F900834609007B
:105DD0003387E60093060002B386E640638C060034
:105DE000B394D40033D7EA003314D600336B970052
:105DF000B399DA00935A040193850A0013050B0046
:105E0000EF00902A1309050093850A00931B0401F3
:105E100013050B00EF00D02493DB0B019304050066
:105E20009305050013850B00EF00D020131909011D
:105E300093D70901B367F900138A040063FEA70032
:105E4000B3878700138AF4FF63E8870063F6A7002F
:105E5000138AE4FFB3878700B384A74093850A00C1
:105E600013850400EF0050241309050093850A00F0
:105E700013850400EF00D01E9399090193040500D7
:105E8000930505001319090113850B0093D9090126
:105E9000EF00501AB36939011386040063FCA900AE
:105EA000B30934011386F4FF63E6890063F4A900A3
:105EB0001386E4FF13140A013364C400130A0000BC
:105EC0006F000013B707000113070001E36CF6EE43
:105ED000130780016FF01FEF138A0600631A060094
:105EE0009305000013051000EF0090171304050040
:105EF000B7070100637EF4129307F00F63F4870085
:105F0000130A8000B35744013309F900034709001D
:105F10009306000233074701B386E64063940612F6
:105F2000B3848440130A1000135B040193050B0033
:105F300013850400EF0050171309050093050B00AB
:105F400013850400931B0401EF00901193DB0B01F8
:105F5000930405009305050013850B00EF00900DD9
:105F60001319090193D70901B367F900938A040053
:105F700063FEA700B3878700938AF4FF63E8870076
:105F800063F6A700938AE4FFB3878700B384A74032
:105F900093050B0013850400EF0010111309050091
:105FA00093050B0013850400EF00900B93990901F2
:105FB00093040500930505001319090113850B00CF
:105FC00093D90901EF001007B36939011386040062
:105FD00063FCA900B30934011386F4FF63E689006A
:105FE00063F4A9001386E4FF13940A013364C40028
:105FF0001305040093050A008320C10203248102D3
:1060000083244102032901028329C101032A81015A
:10601000832A4101032B0101832BC100032C810042
:10602000832C4100032D0100130101036780000050
:10603000B7070001130A0001E366F4EC130A8001BC
:106040006FF05FEC3314D40033DAE400B399DA0074
:1060500033D7EA00935A0401B394D40093850A001D
:1060600013050A00336B9700EF00100413090500B5
:1060700093850A0013050A00931B0401EF00407E7C
:1060800093DB0B01930405009305050013850B00BA
:10609000EF00407A1319090113570B013367E90028
:1060A000138A0400637EA70033078700138AF4FF76
:1060B000636887006376A700138AE4FF33078700CD
:1060C000B304A74093850A0013850400EF00C07D48
:1060D0001309050093850A0013850400EF0040783A
:1060E000930405009305050013850B00EF008074F1
:1060F00013170B011357070113190901B367E900BF
:106100001387040063FEA700B38787001387F4FF9B
:1061100063E8870063F6A7001387E4FFB38787006F
:10612000131A0A01B384A740336AEA006FF0DFDF75
:1061300063ECD51EB707010063F4F6041307F00FF4
:10614000B335D7009395350033D7B60097A7010034
:1061500093874716B387E70003C70700130A0002B7
:106160003307B700330AEA4063160A02130410002B
:10617000E3E096E833B6CA00134416006FF05FE719
:10618000B707000193050001E3E0F6FC93058001E9
:106190006FF09FFBB35CE600B3964601B3ECDC0006
:1061A00033D4E40093DB0C01B397440133D7EA0006
:1061B00093850B0013050400336BF700B3194601F8
:1061C000EF00806E1309050093850B001305040092
:1061D000139C0C01EF00C068135C0C0193040500D4
:1061E0009305050013050C00EF00C06413190901A5
:1061F00013570B013367E90013840400637EA70083
:10620000330797011384F4FF636897016376A7004F
:106210001384E4FF33079701B304A74093850B0071
:1062200013850400EF0040681309050093850B00F7
:1062300013850400EF00C062930405009305050078
:1062400013050C00EF00005F93170B0113190901F0
:1062500093D70701B367F9001386040063FEA70014
:10626000B38797011386F4FF63E8970163F6A700ED
:106270001386E4FFB387970113140401B70B0100E1
:106280003364C4001389FBFF337D240133F92901F2
:10629000B384A7409305090013050D00EF00805952
:1062A000935C040193050900130B050013850C0092
:1062B000EF00405893D90901130C0500938509009C
:1062C00013850C00EF0000571309050093850900A2
:1062D00013050D00EF0000563305850193570B01A0
:1062E0003385A7006374850133097901935705014C
:1062F000B387270163E6F402E392F4BCB707010019
:106300009387F7FF3375F50013150501337BFB0009
:1063100033964A0133056501130A0000E37AA6CCDF
:106320001304F4FF6FF09FB9130A00001304000078
:106330006FF01FCC130101FB23248104232291045D
:10634000232E310323229103232611042320210528
:10635000232C4103232A510323286103232671039D
:10636000232481032320A103232EB101930C0500D4
:10637000938905001304050093840500639E062697
:1063800013090600138A060097AA0100938A8AF26D
:1063900063F4C514B70701006376F6129307F00F94
:1063A00063F4C700130A8000B3574601B38AFA00AA
:1063B00003C70A001305000233074701330AE5400B
:1063C000630C0A00B395490133D7EC003319460139
:1063D000B364B70033944C01935A090193850A00C2
:1063E00013850400EF00404C9309050093850A00D3
:1063F000131B090113850400EF008046135B0B019A
:106400009305050013050B00EF00C04293990901A5
:1064100093570401B3E7F90063FAA700B387270194
:1064200063E6270163F4A700B3872701B384A7407D
:1064300093850A0013850400EF00004793090500C7
:1064400093850A0013850400EF00804113140401B2
:10645000930505009399090113050B0013540401DA
:10646000EF00403D33E48900637AA4003304240143
:10647000636624016374A400330424013304A4403C
:1064800033554401930500008320C1040324810493
:1064900083244104032901048329C103032A8103BE
:1064A000832A4103032B0103832BC102032C8102A6
:1064B000832C4102032D0102832DC101130101052B
:1064C00067800000B7070001130A0001E36EF6ECD5
:1064D000130A80016FF05FED631A06009305000058
:1064E00013051000EF00C03713090500B7070100BE
:1064F000637AF90E9307F00F63F42701130A800003
:10650000B3574901B38AFA0003C70A001305000212
:10651000B384294133074701330AE540E30E0AEA11
:1065200033194901B3DAE900B395490133D7EC00D7
:1065300093540901336BB70013850A009385040057
:10654000EF0080369309050093850400931B090131
:1065500013850A00EF00C03093DB0B0193050500A3
:1065600013850B00EF00002D9399090193570B0140
:10657000B3E7F90033944C0163FAA700B38727010E
:1065800063E6270163F4A700B3872701B38AA74016
:106590009385040013850A00EF000031930905007C
:1065A0009385040013850A00EF00802B93050500F6
:1065B00013850B00EF00002893150B019399090137
:1065C00093D50501B3E5B90063FAA500B3852501AC
:1065D00063E6250163F4A500B3852501B384A540D6
:1065E0006FF09FDFB7070001130A0001E36AF9F0BB
:1065F000130A80016FF0DFF0E3E8D5E8B707010088
:1066000063FCF604930BF00F33B5DB001315350074
:1066100033D7A60097A701009387C7C9B387E700C0
:1066200083CB070093050002B38BAB00338B75411E
:10663000631E0B0263E4360163EACC003384CC4072
:10664000B386D94033B58C00B384A640130504004B
:10665000938504006FF05FE3B707000113050001A5
:10666000E3E8F6FA130580016FF09FFAB39666012E
:10667000335D7601336DDD0033D47901B395690163
:1066800033DC7C0193540D01336CBC001305040012
:1066900093850400B31A6601EF000021130A050078
:1066A000938504001305040033996C01931C0D01BC
:1066B000EF00001B93DC0C0113040500930505009B
:1066C00013850C00EF000017131A0A0113570C0171
:1066D0003367EA00130A0400637EA7003307A701AB
:1066E000130AF4FF6368A7016376A700130AE4FFA7
:1066F0003307A701B309A740938504001385090058
:10670000EF00801A93850400130405001385090027
:10671000EF000015930505009304050013850C0098
:10672000EF00401193150C011314040193D50501DA
:10673000B365B4001387040063FEA500B385A5010B
:106740001387F4FF63E8A50163F6A5001387E4FF50
:10675000B385A501131A0A01B70C0100336AEA00D8
:106760001384FCFFB3778A0033F48A00B384A54016
:1067700013850700930504002326F100135A0A012C
:10678000EF00400B930905009305040013050A0070
:10679000EF00400A13DC0A01930D050093050C007D
:1067A00013050A00EF0000098327C100130A050042
:1067B00093050C0013850700EF00C0073305B501F2
:1067C00013D709013307A7006374B701330A9A018D
:1067D000B70701009387F7FF935507013377F70059
:1067E00013170701B3F7F900B3854501B307F700A5
:1067F00063E6B400639EB400637CF90033865741BE
:10680000B3B7C700B385A541B385F540930706002C
:10681000B307F9403339F900B385B440B385254156
:1068200033947501B3D767013365F400B3D56501BF
:106830006FF09FC5130605001305000093F61500C1
:10684000638406003305C50093D5150013161600A2
:10685000E39605FE678000006340050663C60506F3
:1068600013860500930505001305F0FF630C06026F
:1068700093061000637AB6006358C0001316160022
:1068800093961600E36AB6FE1305000063E6C500A2
:10689000B385C5403365D50093D616001356160050
:1068A000E39606FE6780000093820000EFF05FFB36
:1068B00013850500678002003305A04063D80500FA
:1068C000B305B0406FF0DFF9B305B040938200002C
:1068D000EFF01FF93305A0406780020093820000AB
:1068E00063CA0500634C0500EFF09FF713850500B0
:1068F00067800200B305B040E35805FE3305A040B1
:10690000EFF01FF63305B0406780020097A7010043
:10691000938787C5944317A701001307A7C318439C
:10692000C8C2637BE50017A70100130767C30843CC
:106930008C4391056F90DFC0411122C406C617A792
:106940000100130727C22A8408438C439105EF9066
:106950003FBF97A70100938727BE9C436376F4004F
:1069600097A7010023AA87BCB2402244410182803C
:1069700097A70100938747BF984394437C43FD1733
:106980007CC3FC4299E3736004308280011122CC05
:1069900026CA2A84AE844AC84EC652C456C206CEFF
:1069A000EFB0EFB61C4003290401B7090001B3E5BD
:1069B0009700930AC4000CC08144FD19370A0002F5
:1069C0001840638C2A03032609004A85B3654701F2
:1069D000B376360193175600758F0329490063C4B7
:1069E000070001E7F1BFE39DE6FC9317760063D350
:1069F0000700D58CEFC00FA1E1B793C4F4FFF98C69
:106A000004C0EFB0CFD50840F2406244D2444249BE
:106A1000B249224A924A05618280411106C622C4C7
:106A2000EFE08FD217E7FFFF130787458146054642
:106A30009305400617A501001305C59CEFC01FF183
:106A400019C92A84EFB0AFAD2A8601478146854532
:106A50002285EFC05FFCEFB00F86B24022440145B3
:046A600041018280EE
:02000004800278
:100000006045FEFF5E46FEFF6845FEFF5E46FEFF62
:100010005E46FEFF5E46FEFF5E46FEFF8045FEFF3B
:100020005E46FEFF5E46FEFF9A45FEFFA645FEFFCA
:100030005E46FEFFB845FEFFC445FEFFC445FEFF19
:10004000C445FEFFC445FEFFC445FEFFC445FEFF98
:10005000C445FEFFC445FEFFC445FEFF5E46FEFFED
:100060005E46FEFF5E46FEFF5E46FEFF5E46FEFF0C
:100070005E46FEFF5E46FEFF5E46FEFF5E46FEFFFC
:100080005E46FEFF5E46FEFF5E46FEFF5E46FEFFEC
:100090005E46FEFF5E46FEFF5E46FEFF5E46FEFFDC
:1000A0005E46FEFF5E46FEFF5E46FEFF5E46FEFFCC
:1000B0005E46FEFF5E46FEFF5E46FEFF5E46FEFFBC
:1000C0005E46FEFF5E46FEFF5E46FEFF5E46FEFFAC
:1000D0005E46FEFF5E46FEFF5E46FEFF5E46FEFF9C
:1000E0005E46FEFF5E46FEFF5E46FEFF5E46FEFF8C
:1000F0005E46FEFF5E46FEFF5E46FEFF5E46FEFF7C
:10010000F845FEFF0E46FEFF5E46FEFF5E46FEFF22
:100110005E46FEFF5E46FEFF5E46FEFF5E46FEFF5B
:100120005E46FEFF5446FEFF5E46FEFF5E46FEFF55
:100130000644FEFFBE44FEFF5E46FEFF5E46FEFF37
:10014000F444FEFF5E46FEFF4C45FEFF5E46FEFFAA
:100150005E46FEFF7A45FEFF6C49FEFFC049FEFF8A
:100160007449FEFFC049FEFFC049FEFFC049FEFFC3
:10017000C049FEFF6648FEFFC049FEFFC049FEFFC2
:100180008048FEFF8C48FEFFC049FEFF9E48FEFFF0
:10019000AA48FEFFAA48FEFFAA48FEFFAA48FEFFA3
:1001A000AA48FEFFAA48FEFFAA48FEFFAA48FEFF93
:1001B000AA48FEFFC049FEFFC049FEFFC049FEFF3E
:1001C000C049FEFFC049FEFFC049FEFFC049FEFF17
:1001D000C049FEFFC049FEFFC049FEFFC049FEFF07
:1001E000C049FEFFC049FEFFC049FEFFC049FEFFF7
:1001F000C049FEFFC049FEFFC049FEFFC049FEFFE7
:10020000C049FEFFC049FEFFC049FEFFC049FEFFD6
:10021000C049FEFFC049FEFFC049FEFFC049FEFFC6
:10022000C049FEFFC049FEFFC049FEFFC049FEFFB6
:10023000C049FEFFC049FEFFC049FEFFC049FEFFA6
:10024000C049FEFFC049FEFFC049FEFFC049FEFF96
:10025000C049FEFFC049FEFFDE48FEFF0C49FEFF1D
:10026000C049FEFFC049FEFFC049FEFFC049FEFF76
:10027000C049FEFFC049FEFFC049FEFF6249FEFFC4
:10028000C049FEFFC049FEFFC446FEFFBE47FEFF59
:10029000C049FEFFC049FEFF3048FEFFC049FEFFD7
:1002A0005648FEFFC049FEFFC049FEFFBA49FEFFA7
:1002B000000102020303030304040404040404040D
:1002C00005050505050505050505050505050505DE
:1002D00006060606060606060606060606060606BE
:1002E00006060606060606060606060606060606AE
:1002F000070707070707070707070707070707078E
:10030000070707070707070707070707070707077D
:10031000070707070707070707070707070707076D
:10032000070707070707070707070707070707075D
:10033000080808080808080808080808080808083D
:10034000080808080808080808080808080808082D
:10035000080808080808080808080808080808081D
:10036000080808080808080808080808080808080D
:1003700008080808080808080808080808080808FD
:1003800008080808080808080808080808080808ED
:1003900008080808080808080808080808080808DD
:1003A00008080808080808080808080808080808CD
:1003B000546D725100000000546D7220537663003A
:1003C000286E756C6C2900004572726F7220696E20
:1003D00020787878207461736B73200D0A00000018
:1003E0006D69616F750A00006D69616F75320A0091
:1003F00068756E6772790A0054696D657232000023
:10040000436865636B54696D657200005761697478
:100410004F0000005365744200000000526E647685
:0404200000000000D8
:100424001000000000000000017A5200017C01016C
:100434001B0D02005000000018000000C053FEFF16
:100444005805000000440E507489039406990B81EA
:1004540001880292049305950796089709980A9AC9
:100464000C9B0D036C010AC144C844C944D244D353
:1004740044D444D544D644D744D844D944DA44DB9C
:10048400440E00440B0000004C0000006C0000000F
:10049400C458FEFFDC05000000440E30708903954B
:1004A4000781018802920493059406960897099897
:1004B4000A990B9A0C0370020AC144C844C944D275
:1004C40044D344D444D544D644D744D844D944DA54
:1004D400440E00440B00000050000000BC0000006B
:1004E400505EFEFF0005000000440E50748802892F
:1004F400039305990B810192049406950796089736
:1005040009980A9A0C9B0D0320010AC144C844C9E6
:1005140044D244D344D444D544D644D744D844D90B
:0C05240044DA44DB440E00440B000000ED
:0805C800FC8F01000900000096
:040000058000004037
:00000001FF
